:100000000C9407030C94C4370C94D6030C942D0362
:100010000C942D030C942D030C942D030C942D03A0
:100020000C942D030C942D030C942D030C94C037C9
:100030000C94C2370C942D030C942D030C942D03B7
:100040000C942D030C942D030C942D030C942D0370
:100050000C942D030C942D030C942D030C942D0360
:100060000C942D030C942D0342095D098C106F092B
:100070008C10D3098C108209CC098C108C108C1038
:100080008C108C10E9098C109909A3098C10B20905
:100090008C10E3098C10C209DC098C108C108C10B8
:1000A0008C108C10F909460A560A8C10660A8C10BE
:1000B000CF0A8C10750AC80A8C108C108C108C100A
:1000C0008C10E40A8C10850A950A8C10A50A8C10F5
:1000D000DD0A8C10B40AD60A8C108C108C108C108F
:1000E0008C10EE0A3B0B550B8C10650B8C10290CF9
:1000F0008C10940B1F0C8C108C108C108C108C108E
:10010000410C8C10AD0BC70B8C10D70B8C103A0C1C
:100110008C10060C300C8C108C108C108C108C10E9
:100120004E0C9B0CCF0C8C10E10C8C106F0D8C10B6
:10013000F40C680D8C108C108C108C108C10870DAA
:100140008C10200D300D8C104E0D8C107E0D8C10EF
:10015000580D780D8C108C108C108C108C109C0D00
:10016000E90D100E8C102B0E8C10CC0E8C103A0E4C
:10017000C20E8C108C108C108C108C10E20E8C1017
:10018000520E7E0E8C109B0E8C10DC0E8C10AA0E64
:10019000D20E8C108C108C108C108C10EE0E3B0F2D
:1001A000620F8C107D0F8C1029108C108D0F1F107A
:1001B0008C108C108C108C108C1041108C10A60F91
:1001C000D20F8C10EF0F8C103A108C10FF0F3010E4
:1001D0008C108C108C108C108C104E10C312C3120B
:1001E000D312D312C312C312D312D312C312C31227
:1001F000D312D312D312D312D312D312CA12D012E3
:10020000D312D312CA12D012D312D312CA12D012DE
:10021000D312D312D312D312D312D312C312C312D6
:10022000D312D312C612C612D312D312C812C812D6
:10023000D312D312D312D312D312D312CA12D012A2
:10024000D312D312CA12CC12D312D312CE12D0129E
:10025000A018BB18D11FCD18D11F3219D11FE0181B
:100260002B19D11FD11FD11FD11FD11F4919D11F48
:10027000F7180119D11F1119D11F4219D11F2119C6
:100280003B19D11FD11FD11FD11FD11F5A19AA1934
:10029000BA19D11FCA19D11F331AD11FD9192C1A53
:1002A000D11FD11FD11FD11FD11F481AD11FE9194A
:1002B000F919D11F091AD11F411AD11F181A3A1A58
:1002C000D11FD11FD11FD11FD11F521AA21AB21A8A
:1002D000D11FCC1AD11F4F1BD11FE51A481BD11FAC
:1002E000D11FD11FD11FD11F6A1BD11FF51A051BAA
:1002F000D11F1F1BD11F601BD11F381B591BD11FC2
:10030000D11FD11FD11FD11F771BC71BFB1BD11FB3
:100310000D1CD11F9B1CD11F201C941CD11FD11F51
:10032000D11FD11FD11FB31CD11F4C1C5C1CD11F6E
:100330007A1CD11FAA1CD11F841CA41CD11FD11F41
:10034000D11FD11FD11FC81C181D351DD11F5C1D09
:10035000D11F031ED11F741DFC1DD11FD11FD11F22
:10036000D11FD11F1E1ED11F841DA41DD11FD01D42
:10037000D11F141ED11FE81D0D1ED11FD11FD11F6B
:10038000D11FD11F2B1E7B1E981ED11FBF1ED11F38
:10039000681FD11FD81E611FD11FD11FD11FD11FB0
:1003A000D11F831FD11FE81E081FD11F341FD11F6B
:1003B000791FD11F4D1F721FD11FD11FD11FD11FF8
:1003C000D11F901F1E221E222E222E221E221E22EE
:1003D0002E222E221E221E222E222E222E222E22BD
:1003E0002E222E2225222B222E222E2225222B22A5
:1003F0002E222E2225222B222E222E222E222E2289
:100400002E222E221E221E222E222E2221222122A6
:100410002E222E22232223222E222E222E222E2272
:100420002E222E2225222B222E222E222522272268
:100430002E222E2229222B22D8271428CD2F232802
:10044000CD2F8728CD2F33288328CD2FCD2FCD2F0B
:10045000CD2FCD2F9628CD2F67286E28CD2F75282C
:10046000CD2F9228CD2F7C288E28CD2FCD2FCD2F8C
:10047000CD2FCD2F822FB328BD28CD2F0729CD2FEB
:100480004B2ACD2F5C29442ACD2FCD2FCD2FCD2F18
:10049000CD2F662ACD2F73297D29CD2FCC29CD2FA5
:1004A0005C2ACD2F262A552ACD2FCD2FCD2FCD2F0B
:1004B000CD2F822F842A9F2ACD2FD82ACD2F912B62
:1004C000CD2FF22A8A2BCD2FCD2FCD2FCD2FCD2F73
:1004D000AC2BCD2F092B212BCD2F5C2BCD2FA22B7D
:1004E000CD2F732B9B2BCD2FCD2FCD2FCD2FCD2FC0
:1004F000822FCA2B062CCD2F152CCD2F792CCD2F4A
:10050000252C752CCD2FCD2FCD2FCD2FCD2F882C59
:10051000CD2F592C602CCD2F672CCD2F842CCD2F97
:100520006E2C802CCD2FCD2FCD2FCD2FCD2F822FE8
:10053000A52CAF2CCD2FF92CCD2F4A2ECD2F4E2D03
:10054000362ECD2FCD2FCD2FCD2FCD2F442ECD2FED
:10055000652D6F2DCD2FBE2DCD2F4A2ECD2F182ED0
:100560003D2ECD2FCD2FCD2FCD2FCD2F822F5F2EF6
:100570007A2ECD2FB32ECD2F772FCD2FCD2E632FCB
:10058000CD2FCD2FCD2FCD2FCD2F712FCD2FE42ED1
:10059000FC2ECD2F372FCD2F772FCD2F4D2F6A2F1C
:1005A000CD2FCD2FCD2FCD2FCD2F822F25322832FD
:1005B0002B322E323132343237323A323D324032FF
:1005C000563259325C325F326232653268326B3297
:1005D0006B326E328232853288328B328E32913279
:1005E000943297329A329D32B332B632B932BC323B
:1005F000BF32C232C532C832C832CB320738E937CF
:10060000F6370E382938463858387938903811245A
:100610001FBECFEFD8E0DEBFCDBF14BEA895E0E689
:10062000F0E08081886180838CE0808311E0A0E02D
:10063000B1E0EEE9F9E702C005900D92A230B107F2
:10064000D9F722E0A2E0B1E001C01D92AB3DB207B4
:10065000E1F70E94D2380C94CD3C0C940000A89590
:100660008FE780937D0210928102809181028F3FFB
:1006700021F14A9B04C080917D028F5F03C080916D
:100680007D02815080937D0280917D02811104C0A2
:1006900081E08093A50211C080917D028F3F19F403
:1006A0001092A5020AC026E02A95F1F700C08091B9
:1006B00081028F5F80938102D8CF80917D02882351
:1006C00031F080917D028F3F11F080E0089510920B
:1006D0008500109284008091A502882379F04A99C0
:1006E0000FC080918400909185000397C1F7EDCFF2
:1006F0008091840090918500039739F34A99F8CF4F
:100700008FE780937D0281E0809381028091810256
:100710008F3F21F14B9B04C080917D028F5F03C00E
:1007200080917D02815080937D0280917D028111B4
:1007300004C081E080939C0211C080917D028F3FB4
:1007400019F410929C020AC081EE94E00197F1F72F
:1007500000C00000809181028F5FD6CF80917D0222
:10076000882329F080917D028F3F09F0AECF10924F
:1007700085001092840080919C02882391F04B990F
:1007800012C0809184009091850084399240B9F71D
:100790009CCF80918400909185008439924009F427
:1007A00094CF4B99F6CFA89581E008951F920F92B0
:1007B0000FB60F921124AF92BF92CF92DF92FF92A9
:1007C0000F931F932F933F934F935F936F937F9359
:1007D0008F939F93AF93BF93CF93DF93EF93FF9349
:1007E00080916F00897F80936F00A8958091190197
:1007F0008F5F80931901809119018B30A8F180914E
:10080000990290919A028135910520F120911E0163
:1008100030911F018091990290919A0205972817B3
:10082000390760F020911E0130911F0180919902DB
:1008300090919A0205968217930760F4A89580918B
:100840006000886180936000809160008B7F80935E
:100850006000FFCF1092190180911E0190911F013D
:1008600090939A028093990210921F0110921E0198
:10087000C0917E02C13009F457C250F0C23011F469
:100880000C94F115C33011F40C9426250C94B53555
:10089000909192028091000198133FC2D5E0D093CD
:1008A00000011092920283B1847083B9811110C249
:1008B00086B1817086B9882379F080917E028F5F3E
:1008C00080937E0280917E02843010F010927E022E
:1008D0008AE080930001FCC110927E02D093B602A0
:1008E000C1E0C0939D0246E0A42EA0921001C093E7
:1008F0003501109230015CE3B52EB092270164E11E
:10090000F62EF092050188E790E09093A70280937D
:10091000A60282E380932001C09398027CE8C72E50
:10092000D12CD0928802C0928702C093C00210924C
:1009300093021092B2020EE110E01093A002009315
:100940009F028AE080932F0110931D0100931C01E8
:10095000F092970260919D0286E090E00E94A53C93
:100960006091100188E090E00E94A53C6091350103
:100970008AE090E00E94A53C609130018CE090E01C
:100980000E94A53C609127018EE090E00E94A53C6A
:100990006091050180E190E00E94A53C6091A60273
:1009A0007091A70282E190E00E94B73C6091200123
:1009B00084E190E00E94A53C6091980286E190E07D
:1009C0000E94A53C609187027091880288E190E0C6
:1009D0000E94B73C6091C0028AE190E00E94A53C71
:1009E000609193028CE190E00E94A53C6091B2027C
:1009F0008EE190E00E94A53C60919F027091A00260
:100A000080E290E00E94B73C60912F0182E290E08A
:100A10000E94A53C60911C0170911D0184E290E050
:100A20000E94B73C6091970286E290E00E94A53C4C
:100A3000C093BE02A0929E02C093CF02D0939602B2
:100A4000B092C102F092180186E480930301E4E6BB
:100A5000AE2EB12CB0928C02A0928B02C0938D026C
:100A6000D092D602C092D502C093BF021092CA02A1
:100A70001092AC028FE080933701F4E1CF2ED12C9D
:100A8000D0923201C09231018093C20288E290E09C
:100A90009093800280937F026091BE020E94A53CE9
:100AA00060919E028AE290E00E94A53C6091CF0294
:100AB0008CE290E00E94A53C609196028EE290E06C
:100AC0000E94A53C6091C10280E390E00E94A53C99
:100AD0006091180182E390E00E94A53C60910301BF
:100AE00084E390E00E94A53C60918B0270918C029F
:100AF00086E390E00E94B73C60918D0288E390E02D
:100B00000E94A53C6091D5027091D6028AE390E0E4
:100B10000E94B73C6091BF028CE390E00E94A53C2C
:100B20006091CA028EE390E00E94A53C6091AC0205
:100B300080E490E00E94A53C6091370182E490E05F
:100B40000E94A53C609131017091320184E490E0F3
:100B50000E94B73C6091C20286E490E00E94A53CEE
:100B600060917F027091800288E490E00E94B73C1F
:100B700010921B01D0937C0286E090E09093B1022A
:100B80008093B002C093D4022AE530E03093120182
:100B900020931101109314010093130110939502F7
:100BA00000939402D092AE02C092AD02C0937A023A
:100BB000D093C4029093170180931601C09324012F
:100BC00086E990E09093260180932501B092C602B9
:100BD000A092C5021093860200938502D0922E0146
:100BE000C0922D0160911B018AE490E00E94A53C17
:100BF00060917C028CE490E00E94A53C6091B00280
:100C00007091B1028EE490E00E94B73C6091D402F2
:100C100080E590E00E94A53C609111017091120165
:100C200086E590E00E94B73C609113017091140139
:100C300088E590E00E94B73C609194027091950223
:100C40008AE590E00E94B73C6091AD027091AE02DF
:100C50008CE590E00E94B73C60917A028EE590E0CE
:100C60000E94A53C6091C40280E690E00E94A53CF1
:100C7000609116017091170182E690E00E94B73CE6
:100C80006091240184E690E00E94A53C60912501DA
:100C9000709126018AE690E00E94B73C6091C502FF
:100CA0007091C6028CE690E00E94B73C609185028C
:100CB000709186028EE690E00E94B73C60912D0113
:100CC00070912E0180E790E00E94B73CF092000105
:100CD00086B1817086B9811120C086B1827086B9D3
:100CE000882361F08091B6028F5F8093B602809175
:100CF000B602863078F01092B6020CC08091B6022F
:100D000081508093B6028091B602813F18F085E051
:100D10008093B6028AE080930001809192028F5FF7
:100D2000809392020C94B5359091920280910001CB
:100D300098130C94BB11D5E0D0930001109292024D
:100D400083B1847083B981110FC286B1817086B975
:100D5000882379F080917E028F5F80937E0280915C
:100D60007E02843010F010927E028AE080930001AF
:100D7000FBC110927E02D093B602C0939D0216E092
:100D8000A12EA0921001C0933501109230010CE306
:100D9000B02EB092270184E1F82EF092050188E789
:100DA00090E09093A7028093A60282E380932001B3
:100DB000C09398029CE8C92ED12CD0928802C09290
:100DC0008702C093C002109293021092B2020EE109
:100DD00010E01093A00200939F028AE080932F01FD
:100DE00010931D0100931C01F092970260919D02E7
:100DF00086E090E00E94A53C6091100188E090E0C0
:100E00000E94A53C609135018AE090E00E94A53CDB
:100E1000609130018CE090E00E94A53C6091270138
:100E20008EE090E00E94A53C6091050180E190E099
:100E30000E94A53C6091A6027091A70282E190E019
:100E40000E94B73C6091200184E190E00E94A53CA3
:100E50006091980286E190E00E94A53C6091870233
:100E60007091880288E190E00E94B73C6091C002D6
:100E70008AE190E00E94A53C609193028CE190E0B1
:100E80000E94A53C6091B2028EE190E00E94A53CD8
:100E900060919F027091A00280E290E00E94B73CB6
:100EA00060912F0182E290E00E94A53C60911C01BC
:100EB00070911D0184E290E00E94B73C609197021E
:100EC00086E290E00E94A53CC093BE02A0929E02E2
:100ED000C093CF02D0939602B092C102F092180153
:100EE00086E48093030124E6A22EB12CB0928C02FA
:100EF000A0928B02C0938D02D092D602C092D502EE
:100F0000C093BF021092CA021092AC028FE080938D
:100F1000370134E1C32ED12CD0923201C09231017D
:100F20008093C20288E290E09093800280937F02D7
:100F30006091BE020E94A53C60919E028AE290E010
:100F40000E94A53C6091CF028CE290E00E94A53CFB
:100F5000609196028EE290E00E94A53C6091C102F1
:100F600080E390E00E94A53C6091180182E390E04C
:100F70000E94A53C6091030184E390E00E94A53C9F
:100F800060918B0270918C0286E390E00E94B73CE6
:100F900060918D0288E390E00E94A53C6091D502AB
:100FA0007091D6028AE390E00E94B73C6091BF0244
:100FB0008CE390E00E94A53C6091CA028EE390E031
:100FC0000E94A53C6091AC0280E490E00E94A53CA8
:100FD0006091370182E490E00E94A53C609131016C
:100FE0007091320184E490E00E94B73C6091C202AB
:100FF00086E490E00E94A53C60917F02709180029F
:1010000088E490E00E94B73C10921B01D0937C02D0
:1010100086E090E09093B1028093B002C093D40236
:101020002AE530E03093120120931101109314014E
:10103000009313011093950200939402D092AE0294
:10104000C092AD02C0937A02D093C402909317016C
:1010500080931601C093240186E990E090932601C5
:1010600080932501B092C602A092C5021093860219
:1010700000938502D0922E01C0922D0160911B0138
:101080008AE490E00E94A53C60917C028CE490E0B0
:101090000E94A53C6091B0027091B1028EE490E094
:1010A0000E94B73C6091D40280E590E00E94A53C8C
:1010B000609111017091120186E590E00E94B73CA9
:1010C000609113017091140188E590E00E94B73C93
:1010D00060919402709195028AE590E00E94B73C7D
:1010E0006091AD027091AE028CE590E00E94B73C39
:1010F00060917A028EE590E00E94A53C6091C40266
:1011000080E690E00E94A53C609116017091170165
:1011100082E690E00E94B73C6091240184E690E072
:101120000E94A53C60912501709126018AE690E01D
:101130000E94B73C6091C5027091C6028CE690E0B7
:101140000E94B73C60918502709186028EE690E025
:101150000E94B73C60912D0170912E0180E790E0D4
:101160000E94B73CF092000186B1817086B981116E
:1011700020C086B1827086B9882361F08091B60262
:101180008F5F8093B6028091B602863078F010921D
:10119000B6020CC08091B60281508093B602809155
:1011A000B602813F18F085E08093B6028AE0809312
:1011B000000186B1827086B9811104C08091C3029A
:1011C000806103C08091C3028F7E8093C30286B189
:1011D000847086B9811104C08091C302886003C005
:1011E0008091C302877F8093C30286B1807186B9E4
:1011F000811104C08091C302846003C08091C30246
:101200008B7F8093C30286B1887086B9811104C038
:101210008091C302826003C08091C3028D7F80935E
:10122000C30286B1807286B9811104C08091C30265
:10123000816003C08091C3028E7F8093C30280913E
:10124000B602823009F409C230F4882369F0813093
:1012500009F40EC161C7843009F4ADC408F45DC35C
:10126000853009F4FAC558C7E091C3028E2F90E08B
:10127000FC013197EF31F10508F04EC7EC5CFF4FF0
:101280000C94913C80919D02811104C080911001C9
:101290008E5F03C0809110018F5F80931001909149
:1012A00010018091AF02891720F48091AF028093E2
:1012B00010018AE0809300012FC780919D02815028
:1012C00080939D0280919D02813F10F010929D02BB
:1012D00081E08093CE028AE0809300011DC7809157
:1012E0009D028F5F80939D0280919D02863018F051
:1012F00085E080939D0281E08093CE028AE0809316
:1013000000010AC780919D02811104C080911001E3
:10131000825003C080911001815080931001809110
:101320001001813F10F0109210018AE080930001BB
:10133000F3C69091350181E08927809335018AE0D9
:1013400080930001E9C68091300181508093300183
:1013500080913001813F10F0109230018AE080933B
:101360000001DAC6809130018F5F80933001809157
:101370003001853118F084E1809330018AE0809358
:101380000001CAC69091350181E08927809335011B
:101390008AE080930001C0C681E08093CE028AE09B
:1013A00080930001B9C681E080939D028093CE02B4
:1013B0008AE080930001B0C681E0809335018AE025
:1013C00080930001A9C6109230018AE08093000149
:1013D000A3C686E08093100181E080939D028093F4
:1013E0003501109230018093CE028AE08093000193
:1013F00093C686E08093100181E080939D028093E4
:101400003501109230018093CE029CE39093270126
:1014100094E19093050128E730E03093A7022093F0
:10142000A60222E3209320012CE830E030938802CA
:101430002093870280939802109293028093C002B7
:101440001092B2028093A9022EE130E03093A00204
:1014500020939F028AE080932F0130931D012093F7
:101460001C01909397021092B6029093000154C60B
:10147000E091C3028E2F90E0FC013197EF31F1052E
:1014800008F04AC6ED5AFF4F0C94913C8091270119
:101490008F5F8093270180912701813F18F080EFB3
:1014A000809327018AE08093000136C68091050170
:1014B0008F5F8093050180910501813F18F080EFD7
:1014C000809305018AE08093000126C68091050182
:1014D00081508093050180910501813F10F01092A9
:1014E00005018AE08093000117C680912701815091
:1014F0008093270180912701883018F488E0809339
:1015000027018AE08093000107C680912701865F4A
:101510008093270180912701813F18F080EF80930D
:1015200027018AE080930001F7C5809105018B5F58
:101530008093050180910501813F18F080EF809331
:1015400005018AE080930001E7C58091050185507F
:101550008093050180910501813F10F010920501F3
:101560008AE080930001D8C5809127018A5080933A
:10157000270180912701883020F080912701813F49
:1015800018F088E0809327018AE080930001C4C5A9
:101590008CE3809327018AE080930001BDC584E13C
:1015A000809305018AE080930001B6C58CE38093A7
:1015B00027018AE080930001AFC584E18093050193
:1015C0008AE080930001A8C58CE38093270184E121
:1015D000809305018AE0809300019EC586E0809398
:1015E000100181E080939D028093350110923001BB
:1015F0008093CE029CE39093270194E190930501A0
:1016000028E730E03093A7022093A60222E320933C
:1016100020012CE830E030938802209387028093E9
:101620009802109293028093C0021092B2028093AB
:10163000A9022EE130E03093A00220939F028AE0BD
:1016400080932F0130931D0120931C0190939702EA
:101650001092B602909300015FC5E091C3028E2FF5
:1016600090E0FC013197EF31F10508F055C5EE58D7
:10167000FF4F0C94913C8091A6029091A702019695
:101680009093A7028093A6028091A6029091A70250
:10169000853F914030F084EF91E09093A7028093D2
:1016A000A6028AE08093000137C5809120018F5FF8
:1016B00080932001809120018A3818F089E8809376
:1016C00020018AE08093000127C58091200181508C
:1016D0008093200180912001893118F489E1809361
:1016E00020014AE0409300012091200150912F01F8
:1016F0008091970230E090E0850F911D28173907FF
:101700000CF00AC5809197028150809397028091D6
:1017100097028A3008F000C54093970280912F010C
:10172000815080932F01F8C48091A6029091A70266
:1017300001979093A7028093A6028091A6029091B0
:10174000A7024E9730F48EE190E09093A702809329
:10175000A6028AE080930001DFC48091A6029091E6
:10176000A7020A969093A7028093A6028091A602F0
:101770009091A702853F914030F084EF91E09093E3
:10178000A7028093A6028AE080930001C5C48091DD
:1017900020018B5F80932001809120018A3818F00E
:1017A00089E8809320018AE080930001B5C480918C
:1017B000200185508093200180912001893118F407
:1017C00089E1809320014AE04093000120912001AB
:1017D00050912F018091970230E090E0850F911D8C
:1017E000281739070CF098C4809197028550809390
:1017F0009702809197028A3008F08EC44093970236
:1018000080912F01855080932F0186C48091A6027C
:101810009091A7020A979093A7028093A6028091C5
:10182000A6029091A7024E9730F48EE190E090933B
:10183000A7028093A6028AE0809300016DC488E726
:1018400090E09093A7028093A6028AE08093000123
:1018500063C482E3809320018AE0809300015CC42A
:1018600088E790E09093A7028093A6028AE0809395
:10187000000152C482E3809320018AE0809300013A
:101880004BC488E790E09093A7028093A60282E37E
:10189000809320018AE0809300013EC486E080931B
:1018A000100181E080939D028093350110923001F8
:1018B0008093CE029CE39093270194E190930501DD
:1018C00028E730E03093A7022093A60222E320937A
:1018D00020012CE830E03093880220938702809327
:1018E0009802109293028093C0021092B2028093E9
:1018F000A9022EE130E03093A00220939F028AE0FB
:1019000080932F0130931D0120931C019093970227
:101910001092B60290930001FFC3E091C3028E2F94
:1019200090E0FC013197EF31F10508F0F5C3EF5677
:10193000FF4F0C94913C80919802811106C08091D8
:1019400087029091880288960FC080919802853016
:1019500031F480918702909188020A9605C08091A7
:101960008702909188024496909388028093870220
:101970002091870230918802809133019091340147
:101980008217930740F48091330190913401909332
:101990008802809387028AE080930001BDC3809112
:1019A000980281508093980280919802813F10F0B4
:1019B0001092980281E08093A9028AE0809300014E
:1019C000ABC3809198028F5F8093980280919802B8
:1019D000863018F085E08093980281E08093A90218
:1019E0008AE08093000198C380919802811106C01B
:1019F000809187029091880288970FC08091980209
:101A0000853031F480918702909188020A9705C051
:101A100080918702909188024497909388028093E6
:101A200087028091870290918802893E9D4F20F025
:101A300010928802109287028AE0809300016CC3A2
:101A4000809193028F5F80939302809193028A30FA
:101A50001CF089E0809393028AE0809300015CC3CC
:101A60008091980281110DC08091B202885D8093AF
:101A7000B2028091B202813A08F44EC31092B202CF
:101A80004BC38091B2028C5E8093B2028091B2020D
:101A9000813508F441C31092B2023EC39091C00256
:101AA00081E089278093C0028AE08093000134C3DB
:101AB0008091930281508093930280919302873F9B
:101AC0001CF487EF809393028AE08093000124C383
:101AD00081E08093A9028AE0809300011DC381E028
:101AE000809398028093A9028AE08093000114C336
:101AF000109293028AE0809300010EC381E08093EC
:101B0000C0021092B2028AE08093000105C38CE803
:101B100090E0909388028093870281E080939802FE
:101B2000109293028093C0021092B2028093A90295
:101B30008AE080930001F0C286E08093100181E08A
:101B400080939D0280933501109230018093CE02E4
:101B50009CE39093270194E19093050128E730E0FE
:101B60003093A7022093A60222E3209320012CE8C1
:101B700030E030938802209387028093980210927D
:101B800093028093C0021092B2028093A9022EE1C8
:101B900030E03093A00220939F028AE080932F01CF
:101BA00030931D0120931C01909397021092B6026E
:101BB00090930001B1C2E091C3028E2F90E0FC012E
:101BC0003197EF31F10508F0A7C2E055FF4F0C94B3
:101BD000913C80919F029091A00201969093A00267
:101BE00080939F0280919F029091A00240911C01DE
:101BF00050911D012091A6023091A702840F951FDC
:101C00002817390748F480919F029091A00201970C
:101C10009093A00280939F028AE0809300017CC28F
:101C200080912F018F5F80932F0130912F01809140
:101C300097022091360190E0830F911D30E0281724
:101C400039072CF480912F01815080932F018AE075
:101C50008093000161C280912F01815080932F01F8
:101C600080912F01813F10F010922F018AE0809324
:101C7000000152C280919F029091A002019790931F
:101C8000A00280939F0280919F029091A002893EC2
:101C90009D4F20F01092A00210929F028AE0809344
:101CA00000013AC280919F029091A0020A969093FF
:101CB000A00280939F0280919F029091A002409188
:101CC0001C0150911D012091A6023091A702840FA2
:101CD000951F2817390770F48091A6029091A702EA
:101CE00020911C0130911D01821B930B9093A00247
:101CF00080939F028AE0809300010EC280912F01A1
:101D00008B5F80932F0130912F018091970220915A
:101D1000360190E0830F911D30E0281739073CF41D
:101D20008091360190919702891B80932F018AE060
:101D300080930001F1C180912F01855080932F0184
:101D400080912F01813F10F010922F018AE0809343
:101D50000001E2C180919F029091A0020A979093A6
:101D6000A00280939F0280919F029091A002893EE1
:101D70009D4F20F01092A00210929F028AE0809363
:101D80000001CAC18EE190E09093A00280939F026F
:101D90008AE080930001C0C18AE080932F01809384
:101DA0000001BAC18EE190E09093A00280939F025F
:101DB0008AE080930001B0C18AE080932F01809374
:101DC0000001AAC18EE190E09093A00280939F024F
:101DD0008AE080932F01809300019EC186E080936A
:101DE000100181E080939D028093350110923001B3
:101DF0008093CE029CE39093270194E19093050198
:101E000028E730E03093A7022093A60222E3209334
:101E100020012CE830E030938802209387028093E1
:101E20009802109293028093C0021092B2028093A3
:101E3000A9022EE130E03093A00220939F028AE0B5
:101E400080932F0130931D0120931C0190939702E2
:101E50001092B602909300015FC1E091C3028E2FF1
:101E600090E0FC013197EF31F10508F055C1E153E5
:101E7000FF4F0C94913C80911C0190911D010196A3
:101E800090931D0180931C0180919F029091A0026C
:101E900040911C0150911D012091A6023091A70292
:101EA000840F951F2817390748F480911C019091E1
:101EB0001D01019790931D0180931C018AE080937E
:101EC00000012AC1809197028F5F80939702309121
:101ED0002F01809197022091360190E0830F911D90
:101EE00030E0281739072CF48091970281508093B5
:101EF00097028AE0809300010FC180919702815080
:101F000080939702809197028A3018F48AE0809338
:101F100097028AE080930001FFC080911C0190919C
:101F20001D01019790931D0180931C0180911C015C
:101F300090911D010F9730F48FE090E090931D0178
:101F400080931C018AE080930001E6C080911C010F
:101F500090911D010A9690931D0180931C01809120
:101F60009F029091A00240911C0150911D0120916F
:101F7000A6023091A702840F951F2817390770F425
:101F80008091A6029091A70220919F023091A00219
:101F9000821B930B90931D0180931C018AE0809318
:101FA0000001BAC0809197028B5F809397023091B5
:101FB0002F01809197022091360190E0830F911DAF
:101FC00030E0281739073CF48091360190912F01B9
:101FD000891B809397028AE0809300019DC08091C5
:101FE0009702855080939702809197028A3018F467
:101FF0008AE0809397028AE0809300018DC08091EF
:102000001C0190911D010A9790931D0180931C0162
:1020100080911C0190911D010F9738F080911C0157
:1020200090911D01893E9D4F30F08FE090E090939C
:102030001D0180931C018AE0809300016DC08EE138
:1020400090E090931D0180931C018AE08093000131
:1020500063C084E1809397028AE0809300015CC0B2
:102060008EE190E090931D0180931C018AE08093A3
:10207000000152C084E1809397028AE080930001BE
:102080004BC08EE190E090931D0180931C0184E190
:10209000809397028AE0809300013EC086E080939F
:1020A000100181E080939D028093350110923001F0
:1020B0008093CE029CE39093270194E190930501D5
:1020C00028E730E03093A7022093A60222E3209372
:1020D00020012CE830E0309388022093870280931F
:1020E0009802109293028093C0021092B2028093E1
:1020F000A9022EE130E03093A00220939F028AE0F3
:1021000080932F0130931D0120931C01909397021F
:102110001092B6029093000180919F029091A002CC
:1021200040911C0150911D012091A6023091A702FF
:10213000840F951F28173907D8F58091A602909132
:10214000A70220919F023091A002821B930B9093D3
:102150001D0180931C0180911C0190911D01893EFD
:102160009D4F30F480911C0190911D010F9700F557
:102170008FE090E090931D0180931C0180919F025D
:102180009091A00240911C0150911D012091A60246
:102190003091A702840F951F2817390748F48091C2
:1021A000A6029091A7020F979093A00280939F029E
:1021B000809105012091200190E0820F911D820FF6
:1021C000911D8331914054F02091050182E191E00D
:1021D000821B91099595879580932001809120011C
:1021E00090913001891B809336018091200190915C
:1021F0003001890F8093B30230912F0180919702B3
:102200002091360190E0830F911D30E028173907A7
:1022100064F58091360120912F0190E0821B910995
:102220009093A4028093A3028091A3029091A402B0
:10223000809397028091A3029091A4020A97ACF434
:102240008AE08093970230912F018091970220912C
:10225000360190E0830F911D30E0281739072CF4E8
:10226000809136018A5080932F0180919D028230A7
:1022700081F030F4882359F0813091F48CE00EC065
:10228000843059F040F0853059F484E007C088E18B
:1022900005C088E003C086E001C085E08093AF02FE
:1022A0008091CE028130D9F480919D02823081F0FC
:1022B00030F4882359F0813081F486E00CC08430FA
:1022C00049F040F0853049F482E005C08CE003C05D
:1022D00084E001C083E0809310011092CE028091CF
:1022E0009802823099F038F4882369F08130D1F473
:1022F00088E191E013C0843079F058F0853091F492
:1023000088E290E00BC080EE91E008C088EC90E09D
:1023100005C088E790E002C080E590E0909334012A
:10232000809333018091A902813029F58091980230
:10233000823099F038F4882369F08130D1F48CE848
:1023400090E013C0843079F058F0853091F484E146
:1023500090E00BC080EF90E008C084E690E005C0FC
:102360008CE390E002C088E290E090938802809332
:1023700087021092A902809192028F5F809392024D
:1023800080919B028F5F80939B0290919B02809132
:10239000AF02981710F010929B0290919B028091CF
:1023A0001001981710F481E001C082E080932A01A7
:1023B0008091D7029091D80201969093D802809391
:1023C000D7024091D7025091D80280913301909169
:1023D00034012091B202820F911D820F911D481786
:1023E000590720F01092D8021092D7022091D702FC
:1023F0003091D8028091870290918802281739077E
:1024000010F481E01FC02091D7023091D802809152
:102410008702909188024091B202840F911D281783
:10242000390798F02091D7023091D802809133017A
:10243000909134014091B202840F911D2817390701
:1024400020F482E080930A0102C010920A012091D8
:1024500027018091A6029091A702820F911D90936F
:102460008A02809389028091270190E0909329014C
:102470008093280180910A01823081F440912701E4
:1024800020919F023091A00280919302082E000CAF
:10249000990B840F911D820F931F08C02091270173
:1024A00080919F029091A002820F911D9093230131
:1024B00080932201809122019091230120911C019F
:1024C00030911D01820F931F9093DA028093D902FD
:1024D00020912201309123018091270190E028175B
:1024E000390738F08091220190912301893E9D4F58
:1024F00038F08091270190E090932301809322018E
:102500002091D9023091DA028091890290918A0259
:102510008217930740F48091890290918A029093E8
:10252000DA028093D9028091200120912F019091AD
:102530009702920F891B8093C8022091C0023091AC
:10254000350190910A0180912A0160E2269FA00145
:10255000112460E1369F90011124242B282B34E0B4
:10256000939FC0011124822B8093C902E091C9027C
:102570008E2F90E0FC013197EA33F105A0F4E2518F
:10258000FF4F0C94913C10927B020DC080E209C079
:1025900082E007C080E105C081E203C082E101C0A2
:1025A00081E080937B0280917B02803109F403C13A
:1025B00048F48130A1F0823011F00C94B5351092BE
:1025C000810267C0803209F400C2813209F457C227
:1025D000823111F00C94B5351092810246C11092EF
:1025E000810290918102809105019817A8F4809151
:1025F0001E0190911F019C012F5F3F4F30931F01DF
:1026000020931E01FC01E75CFE4F10828091810245
:102610008F5F80938102E5CF1092810290918102B9
:102620008091B3029817A8F480911E0190911F0128
:102630009C012F5F3F4F30931F0120931E01FC012F
:10264000E75CFE4F1082809181028F5F8093810250
:10265000E5CF1092810221E09091810280913601B4
:10266000981710F00C94B53580911E0190911F01C0
:10267000AC014F5F5F4F50931F0140931E01FC015F
:10268000E75CFE4F2083809181028F5F80938102FF
:10269000E3CF90918102809105019817A8F4809171
:1026A0001E0190911F019C012F5F3F4F30931F012E
:1026B00020931E01FC01E75CFE4F10828091810295
:1026C0008F5F80938102E5CF109281029091810209
:1026D000809120019817A8F480911E0190911F010C
:1026E0009C012F5F3F4F30931F0120931E01FC017F
:1026F000E75CFE4F1082809181028F5F80938102A0
:10270000E5CF10928102909181028091300198175B
:10271000A8F480911E0190911F019C012F5F3F4FF3
:1027200030931F0120931E01FC01E75CFE4F1082D5
:10273000809181028F5F80938102E5CF10928102A8
:102740009091810280912F019817A8F480911E0129
:1027500090911F019C012F5F3F4F30931F012093E9
:102760001E01FC01E75CFE4F1082809181028F5FA9
:1027700080938102E5CF1092810222E09091810244
:1027800080919702981710F00C94B53580911E0136
:1027900090911F01AC014F5F5F4F50931F01409319
:1027A0001E01FC01E75CFE4F2083809181028F5F58
:1027B00080938102E3CF10928102909181028091F7
:1027C00005019817A8F480911E0190911F019C01AA
:1027D0002F5F3F4F30931F0120931E01FC01E75CE8
:1027E000FE4F1082809181028F5F80938102E5CF3E
:1027F0001092810221E09091810280913601981718
:10280000A8F480911E0190911F01AC014F5F5F4FB2
:1028100050931F0140931E01FC01E75CFE4F208393
:10282000809181028F5F80938102E5CF10928102B7
:10283000909181028091B302981710F00C94B535F5
:1028400080911E0190911F019C012F5F3F4F30939B
:102850001F0120931E01FC01E75CFE4F1082809156
:1028600081028F5F80938102E3CF909181028091FA
:1028700005019817A8F480911E0190911F019C01F9
:102880002F5F3F4F30931F0120931E01FC01E75C37
:10289000FE4F1082809181028F5F80938102E5CF8D
:1028A0001092810221E09091810280913601981767
:1028B000A8F480911E0190911F01AC014F5F5F4F02
:1028C00050931F0140931E01FC01E75CFE4F2083E3
:1028D000809181028F5F80938102E5CF1092810207
:1028E00090918102809130019817A8F480911E0187
:1028F00090911F019C012F5F3F4F30931F01209348
:102900001E01FC01E75CFE4F1082809181028F5F07
:1029100080938102E5CF1092810290918102809193
:1029200030019817A8F480911E0190911F019C011D
:102930002F5F3F4F30931F0120931E01FC01E75C86
:10294000FE4F1082809181028F5F80938102E5CFDC
:10295000109281029091810280912F019817A8F422
:1029600080911E0190911F019C012F5F3F4F30937A
:102970001F0120931E01FC01E75CFE4F1082809135
:1029800081028F5F80938102E5CF1092810222E065
:102990009091810280919702981710F00C94B535B0
:1029A00080911E0190911F01AC014F5F5F4F5093CA
:1029B0001F0140931E01FC01E75CFE4F20838091C4
:1029C00081028F5F80938102E3CF10928102909108
:1029D0008102809105019817A8F480911E019091C1
:1029E0001F019C012F5F3F4F30931F0120931E0159
:1029F000FC01E75CFE4F1082809181028F5F809323
:102A00008102E5CF109281029091810280912F0185
:102A10009817A8F480911E0190911F019C012F5FCF
:102A20003F4F30931F0120931E01FC01E75CFE4FD6
:102A30001082809181028F5F80938102E5CF109296
:102A4000810222E09091810280919702981710F004
:102A50000C94B53580911E0190911F01AC014F5F20
:102A60005F4F50931F0140931E01FC01E75CFE4F36
:102A70002083809181028F5F80938102E3CF109247
:102A8000810290918102809105019817A8F48091AC
:102A90001E0190911F019C012F5F3F4F30931F013A
:102AA00020931E01FC01E75CFE4F108280918102A1
:102AB0008F5F80938102E5CF109281029091810215
:102AC00080912F019817A8F480911E0190911F0109
:102AD0009C012F5F3F4F30931F0120931E01FC018B
:102AE000E75CFE4F1082809181028F5F80938102AC
:102AF000E5CF1092810222E09091810280919702AD
:102B00009817A8F480911E0190911F01AC014F5FAE
:102B10005F4F50931F0140931E01FC01E75CFE4F85
:102B20002083809181028F5F80938102E5CF109294
:102B30008102909181028091C8029817A8F4809137
:102B40001E0190911F019C012F5F3F4F30931F0189
:102B500020931E01FC01E75CFE4F108280918102F0
:102B60008F5F80938102E5CF109281029091810264
:102B7000809130019817A8F480911E0190911F0157
:102B80009C012F5F3F4F30931F0120931E01FC01DA
:102B9000E75CFE4F1082809181028F5F80938102FB
:102BA000E5CF1092810221E090918102809136015F
:102BB000981710F00C94B53580911E0190911F016B
:102BC000AC014F5F5F4F50931F0140931E01FC010A
:102BD000E75CFE4F2083809181028F5F80938102AA
:102BE000E3CF909192028091000198130C940721F9
:102BF000D5E0D09300011092920283B1847083B922
:102C0000811110C286B1817086B9882379F08091D4
:102C10007E028F5F80937E0280917E02843010F06E
:102C200010927E028AE080930001FCC110927E0225
:102C3000D093B602C1E0C0939D0266E0A62EA0929A
:102C40001001C0933501109230017CE3B72EB09291
:102C50002701E4E1FE2EF092050188E790E09093D1
:102C6000A7028093A60282E380932001C09398027A
:102C7000FCE8CF2ED12CD0928802C0928702C0935C
:102C8000C002109293021092B2020EE110E0109373
:102C9000A00200939F028AE080932F0110931D01F0
:102CA00000931C01F092970260919D0286E090E0F3
:102CB0000E94A53C6091100188E090E00E94A53C34
:102CC000609135018AE090E00E94A53C609130015E
:102CD0008CE090E00E94A53C609127018EE090E09E
:102CE0000E94A53C6091050180E190E00E94A53C16
:102CF0006091A6027091A70282E190E00E94B73C29
:102D00006091200184E190E00E94A53C60919802CE
:102D100086E190E00E94A53C609187027091880254
:102D200088E190E00E94B73C6091C0028AE190E0A7
:102D30000E94A53C609193028CE190E00E94A53C2A
:102D40006091B2028EE190E00E94A53C60919F02EA
:102D50007091A00280E290E00E94B73C60912F0148
:102D600082E290E00E94A53C60911C0170911D01DF
:102D700084E290E00E94B73C6091970286E290E086
:102D80000E94A53CC093BE02A0929E02C093CF02B7
:102D9000D0939602B092C102F092180186E480931B
:102DA0000301A4E6AA2EB12CB0928C02A0928B0251
:102DB000C0938D02D092D602C092D502C093BF02BA
:102DC0001092CA021092AC028FE080933701B4E1F6
:102DD000CB2ED12CD0923201C09231018093C2020D
:102DE00088E290E09093800280937F026091BE021F
:102DF0000E94A53C60919E028AE290E00E94A53C60
:102E00006091CF028CE290E00E94A53C6091960216
:102E10008EE290E00E94A53C6091C10280E390E0C8
:102E20000E94A53C6091180182E390E00E94A53CBD
:102E30006091030184E390E00E94A53C60918B02C5
:102E400070918C0286E390E00E94B73C60918D0205
:102E500088E390E00E94A53C6091D5027091D60273
:102E60008AE390E00E94B73C6091BF028CE390E05F
:102E70000E94A53C6091CA028EE390E00E94A53CAE
:102E80006091AC0280E490E00E94A53C6091370123
:102E900082E490E00E94A53C609131017091320182
:102EA00084E490E00E94B73C6091C20286E490E026
:102EB0000E94A53C60917F027091800288E490E0BE
:102EC0000E94B73C10921B01D0937C0286E090E0F8
:102ED0009093B1028093B002C093D4022AE530E00F
:102EE00030931201209311011093140100931301E8
:102EF0001093950200939402D092AE02C092AD025C
:102F0000C0937A02D093C402909317018093160164
:102F1000C093240186E990E09093260180932501D7
:102F2000B092C602A092C502109386020093850259
:102F3000D0922E01C0922D0160911B018AE490E095
:102F40000E94A53C60917C028CE490E00E94A53C2C
:102F50006091B0027091B1028EE490E00E94B73CA3
:102F60006091D40280E590E00E94A53C609111013F
:102F70007091120186E590E00E94B73C60911301C8
:102F80007091140188E590E00E94B73C6091940232
:102F9000709195028AE590E00E94B73C6091AD0285
:102FA0007091AE028CE590E00E94B73C60917A028D
:102FB0008EE590E00E94A53C6091C40280E690E01E
:102FC0000E94A53C609116017091170182E690E085
:102FD0000E94B73C6091240184E690E00E94A53CE9
:102FE00060912501709126018AE690E00E94B73C2D
:102FF0006091C5027091C6028CE690E00E94B73CD9
:1030000060918502709186028EE690E00E94B73C46
:1030100060912D0170912E0180E790E00E94B73CF5
:10302000F092000186B1817086B9811120C086B10D
:10303000827086B9882361F08091B6028F5F809399
:10304000B6028091B602863078F01092B6020CC0BB
:103050008091B60281508093B6028091B602813F82
:1030600018F085E08093B6028AE08093000186B173
:10307000827086B9811104C08091C302806103C04F
:103080008091C3028F7E8093C30286B1847086B91B
:10309000811104C08091C302886003C08091C30283
:1030A000877F8093C30286B1807186B9811104C085
:1030B0008091C302846003C08091C3028B7F8093A0
:1030C000C30286B1887086B9811104C08091C302A1
:1030D000826003C08091C3028D7F8093C30286B15A
:1030E000807286B9811104C08091C302816003C0DF
:1030F0008091C3028E7F8093C3028091B60282309A
:1031000009F412C230F4882369F0813009F414C143
:1031100048C7843009F47EC408F42BC3853009F411
:10312000DCC53FC7E091C3028E2F90E0FC013197D0
:10313000EF31F10508F035C7E85DFE4F0C94913C86
:103140008091BE02811104C080919E028E5F03C0F7
:1031500080919E028F5F80939E0290919E0280914B
:103160000401891720F48091040180939E028AE073
:103170008093000116C78091BE0281508093BE02E9
:103180008091BE02813F10F01092BE0281E08093D8
:10319000BA028AE08093000104C78091BE028F5F6B
:1031A0008093BE028091BE02863018F085E0809345
:1031B000BE0281E08093BA028AE080930001F1C6EA
:1031C0008091BE02811104C080919E02825003C092
:1031D00080919E02815080939E0280919E02813F49
:1031E00010F010929E028AE080930001DAC690915E
:1031F000CF0281E089278093CF028AE0809300018B
:10320000D0C680919602815080939602809196025A
:10321000853018F485E0809396028AE0809300015F
:10322000C0C6809196028F5F80939602809196022D
:10323000893218F088E2809396028AE08093000138
:10324000B0C69091CF0281E089278093CF028AE0B7
:1032500080930001A6C681E08093BA028AE0809341
:1032600000019FC681E08093BE028093BA028AE08B
:103270008093000196C681E08093CF028AE080931C
:1032800000018FC685E0809396028AE0809300015A
:1032900088C686E080939E0281E08093BE02809380
:1032A000CF0295E0909396028093BA028AE08093D1
:1032B000000177C686E080939E0281E08093BE0283
:1032C0008093CF0295E0909396028093BA029CE39C
:1032D0009093C10294E19093180126E42093030196
:1032E00024E630E030938C0220938B022CE830E00F
:1032F0003093D6022093D50280938D021092CA0299
:103300008093BF021092AC0280930F018FE08093F4
:10331000370124E130E03093320120933101809372
:10332000C20228E230E03093800220937F021092A4
:10333000B6029093000135C6E091C3028E2F90E053
:10334000FC013197EF31F10508F02BC6E95BFE4F28
:103350000C94913C8091C1028F5F8093C102809157
:10336000C102813F18F080EF8093C1028AE0809310
:10337000000117C6809118018F5F8093180180911A
:103380001801813F18F080EF809318018AE0809344
:10339000000107C680911801815080931801809127
:1033A0001801813F10F0109218018AE0809300010B
:1033B000F8C58091C10281508093C1028091C10201
:1033C000883018F488E08093C1028AE0809300017D
:1033D000E8C58091C102865F8093C1028091C102DD
:1033E000813F18F080EF8093C1028AE08093000152
:1033F000D8C580911801865F8093180180911801CB
:10340000813F18F080EF809318018AE080930001DB
:10341000C8C5809118018A508093180180911801C5
:10342000813F10F0109218018AE080930001B9C525
:103430008091C1028A508093C1028091C10288307C
:1034400020F08091C102813F18F088E08093C10292
:103450008AE080930001A5C58CE38093C1028AE0D5
:10346000809300019EC584E1809318018AE08093D7
:10347000000197C58CE38093C1028AE0809300012C
:1034800090C584E1809318018AE08093000189C58A
:103490008CE38093C10284E1809318018AE08093D9
:1034A00000017FC586E080939E0281E08093BE028A
:1034B0008093CF0295E0909396028093BA029CE3AA
:1034C0009093C10294E19093180126E420930301A4
:1034D00024E630E030938C0220938B022CE830E01D
:1034E0003093D6022093D50280938D021092CA02A7
:1034F0008093BF021092AC0280930F018FE0809303
:10350000370124E130E03093320120933101809380
:10351000C20228E230E03093800220937F021092B2
:10352000B602909300013DC5E091C3028E2F90E05A
:10353000FC013197EF31F10508F033C5EA59FE4F30
:103540000C94913C809103018F5F809303018091E3
:1035500003018B3F18F08AEF809303018AE0809388
:1035600000011FC580918B0290918C02019690936F
:103570008C0280938B0280918B0290918C0283311C
:10358000914030F082E191E090938C0280938B0225
:103590008AE08093000105C580918B0290918C0296
:1035A000019790938C0280938B0280918B02909173
:1035B0008C02C29730F482E390E090938C02809367
:1035C0008B028AE080930001ECC48091030181505A
:1035D00080930301809103018C3318F48CE3809372
:1035E00003018AE080930001DCC4809103018B5FBA
:1035F00080930301809103018B3F18F08AEF809341
:1036000003018AE080930001CCC480918B029091E9
:103610008C020A9690938C0280938B0280918B028D
:1036200090918C028331914030F082E191E090934F
:103630008C0280938B028AE080930001B2C4809157
:103640008B0290918C020A9790938C0280938B024C
:1036500080918B0290918C02C29730F482E390E0CB
:1036600090938C0280938B028AE08093000199C42E
:1036700080910301855080930301809103018C3375
:1036800018F48CE3809303018AE08093000189C4DD
:1036900086E4809303018AE08093000182C484E67B
:1036A00090E090938C0280938B028AE080930001DB
:1036B00078C486E4809303018AE08093000171C49A
:1036C00084E690E090938C0280938B028AE0809352
:1036D000000167C486E48093030184E690E0909340
:1036E0008C0280938B028AE0809300015AC486E0AA
:1036F00080939E0281E08093BE028093CF0295E08A
:10370000909396028093BA029CE39093C10294E155
:103710009093180126E42093030124E630E03093CF
:103720008C0220938B022CE830E03093D602209359
:10373000D50280938D021092CA028093BF0210922C
:10374000AC0280930F018FE08093370124E130E0D9
:1037500030933201209331018093C20228E230E09D
:103760003093800220937F021092B6029093000162
:1037700018C4E091C3028E2F90E0FC013197EF3125
:10378000F10508F00EC4EB57FE4F0C94913C80916C
:103790008D02811106C08091D5029091D602889643
:1037A0000FC080918D02853031F48091D5029091C7
:1037B000D6020A9605C08091D5029091D602449611
:1037C0009093D6028093D5022091D5023091D602F3
:1037D0008091D0029091D1028217930740F480919A
:1037E000D0029091D1029093D6028093D5028AE0C4
:1037F00080930001D6C380918D02815080938D0209
:1038000080918D02813F10F010928D0281E08093B3
:103810000F018AE080930001C4C380918D028F5F05
:1038200080938D0280918D02863018F085E0809320
:103830008D0281E080930F018AE080930001B1C383
:1038400080918D02811106C08091D5029091D6029F
:1038500088970FC080918D02853031F48091D50218
:103860009091D6020A9705C08091D5029091D60218
:1038700044979093D6028093D5028091D50290917F
:10388000D602893E9D4F20F01092D6021092D502AA
:103890008AE08093000185C38091CA028F5F809384
:1038A000CA028091CA028A301CF089E08093CA0261
:1038B0008AE08093000175C380918D0281110DC053
:1038C0008091AC02885D8093AC028091AC02813A19
:1038D00008F467C31092AC0264C38091AC028C5EA2
:1038E0008093AC028091AC02813508F45AC31092E7
:1038F000AC0257C39091BF0281E089278093BF0239
:103900008AE0809300014DC38091CA028150809368
:10391000CA028091CA02873F1CF487EF8093CA02D3
:103920008AE0809300013DC381E080930F018AE02B
:103930008093000136C381E080938D0280930F0154
:103940008AE0809300012DC31092CA028AE080931E
:10395000000127C381E08093BF021092AC028AE08D
:10396000809300011EC38CE890E09093D602809370
:10397000D50281E080938D021092CA028093BF022B
:103980001092AC0280930F018AE08093000109C37A
:1039900086E080939E0281E08093BE028093CF02F6
:1039A00095E0909396028093BA029CE39093C102B3
:1039B00094E19093180126E42093030124E630E07B
:1039C00030938C0220938B022CE830E03093D602A7
:1039D0002093D50280938D021092CA028093BF0279
:1039E0001092AC0280930F018FE08093370124E1A5
:1039F00030E030933201209331018093C20228E2FB
:103A000030E03093800220937F021092B6029093B0
:103A10000001C7C2E091C3028E2F90E0FC013197F4
:103A2000EF31F10508F0BDC2EC55FE4F0C94913C0E
:103A3000809137018F5F8093370120912101409160
:103A400037018091C20230E02450310990E0840FA8
:103A5000911D821793072CF080913701815080933C
:103A600037018AE0809300019CC2809131019091DE
:103A7000320101969093320180933101809131019E
:103A80009091320140917F025091800220918B02EF
:103A900030918C02840F951F2817390748F48091C4
:103AA000310190913201019790933201809331015D
:103AB0008AE08093000175C28091310190913201BA
:103AC000019790933201809331018091310190915F
:103AD0003201893E9D4F20F0109232011092310147
:103AE0008AE0809300015DC280913701815080930C
:103AF000370180913701853018F485E080933701D4
:103B00008AE0809300014DC280913701865F8093E7
:103B1000370120912101409137018091C20230E0AC
:103B20002450310990E0840F911D8217930744F0CF
:103B3000809121019091C2028550891B80933701A9
:103B40008AE0809300012DC2809131019091320171
:103B50000A969093320180933101809131019091C6
:103B6000320140917F025091800220918B0230916E
:103B70008C02840F951F2817390770F480918B02EF
:103B800090918C0220917F0230918002821B930BD6
:103B900090933201809331018AE08093000101C249
:103BA00080913101909132010A9790933201809374
:103BB00031018091310190913201893E9D4F20F079
:103BC00010923201109231018AE080930001E9C124
:103BD000809137018A508093370180913701853079
:103BE00020F080913701813F18F085E08093370104
:103BF0008AE080930001D5C18FE0809337018AE08D
:103C000080930001CEC184E190E0909332018093D3
:103C100031018AE080930001C4C18FE080933701B5
:103C20008AE080930001BDC184E190E0909332016D
:103C3000809331018AE080930001B3C18FE08093CB
:103C4000370184E190E090933201809331018AE062
:103C500080930001A6C186E080939E0281E080935C
:103C6000BE028093CF0295E0909396028093BA02B1
:103C70009CE39093C10294E19093180126E4209371
:103C8000030124E630E030938C0220938B022CE871
:103C900030E03093D6022093D50280938D021092AB
:103CA000CA028093BF021092AC0280930F018FE092
:103CB0008093370124E130E03093320120933101C9
:103CC0008093C20228E230E03093800220937F028A
:103CD0001092B6029093000164C1E091C3028E2F4E
:103CE00090E0FC013197EF31F10508F05AC1ED5336
:103CF000FE4F0C94913C8091C2028F5F8093C20270
:103D000020912101409137018091C20230E024507E
:103D1000310990E0840F911D821793072CF0809158
:103D2000C20281508093C2028AE08093000139C1AF
:103D300080917F02909180020196909380028093FF
:103D40007F02809131019091320140917F02509128
:103D5000800220918B0230918C02840F951F2817CE
:103D6000390748F480917F029091800201979093E7
:103D7000800280937F028AE08093000112C18091CB
:103D80007F029091800201979093800280937F023E
:103D900080917F0290918002449730F484E190E01A
:103DA0009093800280937F028AE080930001F9C0A3
:103DB0008091C20281508093C2028091C2028A30F7
:103DC00018F48AE08093C2028AE080930001E9C07F
:103DD0008091C202865F8093C202209121014091AE
:103DE00037018091C20230E02450310990E0840F05
:103DF000911D8217930744F0809121019091370122
:103E00008550891B8093C2028AE080930001C9C05B
:103E100080917F02909180020A9690938002809315
:103E20007F02809131019091320140917F02509147
:103E3000800220918B0230918C02840F951F2817ED
:103E4000390770F480918B0290918C02209131019E
:103E500030913201821B930B9093800280937F02FA
:103E60008AE0809300019DC080917F029091800242
:103E70000A979093800280937F0280917F029091B5
:103E80008002449730F484E190E090938002809324
:103E90007F028AE08093000184C08091C2028A5030
:103EA0008093C2028091C2028A3020F08091C202C7
:103EB000813F18F08AE08093C2028AE0809300017B
:103EC00070C08FE08093C2028AE08093000169C0D5
:103ED00088E290E09093800280937F028AE0809352
:103EE00000015FC08FE08093C2028AE080930001EE
:103EF00058C088E290E09093800280937F028AE02D
:103F0000809300014EC08FE08093C20288E290E06F
:103F10009093800280937F028AE08093000141C0E9
:103F200086E080939E0281E08093BE028093CF0260
:103F300095E0909396028093BA029CE39093C1021D
:103F400094E19093180126E42093030124E630E0E5
:103F500030938C0220938B022CE830E03093D60211
:103F60002093D50280938D021092CA028093BF02E3
:103F70001092AC0280930F018FE08093370124E10F
:103F800030E030933201209331018093C20228E265
:103F900030E03093800220937F021092B60290931B
:103FA00000018091030190919602891B8093210169
:103FB00020912101409137018091C20230E02450CC
:103FC000310990E0840F911D8217930794F180913D
:103FD00021012091370190E00597821B9109909370
:103FE000910280939002809190029091910280932F
:103FF000C20280919002909191020A97D4F48AE0D3
:104000008093C20220912101409137018091C20228
:1040100030E02450310990E0840F911D82179307FE
:1040200044F0809121019091C2028550891B8093B8
:104030003701809131019091320140917F0250917E
:10404000800220918B0230918C02840F951F2817DB
:10405000390708F041C080918B0290918C02209129
:10406000310130913201821B930B9093B502809302
:10407000B4028091B4029091B50290938002809333
:104080007F028091B4029091B50244972CF584E1AF
:1040900090E09093800280937F0280913101909113
:1040A000320140917F025091800220918B02309129
:1040B0008C02840F951F2817390770F480918B02AA
:1040C00090918C0220917F0230918002821B930B91
:1040D00090933201809331012091180180918B02DD
:1040E00090918C02820F911D8331914050F020916C
:1040F000180182E191E0821B910990938C028093D8
:104100008B028091BE02823081F030F4882359F016
:10411000813091F48CE00EC0843059F040F085304D
:1041200059F484E007C088E105C088E003C086E058
:1041300001C085E0809304018091BA028130D9F4F6
:104140008091BE02823081F030F4882359F08130B2
:1041500081F486E00CC0843049F040F0853049F4A9
:1041600082E005C08CE003C084E001C083E080935E
:104170009E021092BA0280918D02823099F038F43A
:10418000882369F08130D1F488E191E013C0843054
:1041900079F058F0853091F488E290E00BC080EE21
:1041A00091E008C088EC90E005C088E790E002C08C
:1041B00080E590E09093D1028093D00280910F012E
:1041C000813029F580918D02823099F038F488236E
:1041D00069F08130D1F48CE890E013C0843079F03C
:1041E00058F0853091F484E190E00BC080EF90E0CE
:1041F00008C084E690E005C08CE390E002C088E24D
:1042000090E09093D6028093D50210920F01809196
:1042100092028F5F80939202809184028F5F8093DD
:1042200084029091840280910401981710F01092FA
:1042300084029091840280919E02981710F481E08C
:1042400001C082E08093A1028091B8029091B902EE
:1042500001969093B9028093B8024091B8025091B0
:10426000B9028091D0029091D1022091AC02820FCC
:10427000911D820F911D4817590720F01092B90225
:104280001092B8022091B8023091B9028091D50203
:104290009091D6022817390710F481E01FC02091B1
:1042A000B8023091B9028091D5029091D602409126
:1042B000AC02840F911D2817390798F02091B8029D
:1042C0003091B9028091D0029091D1024091AC021C
:1042D000840F911D2817390720F482E08093BC02D7
:1042E00002C01092BC028091A102823029F4809118
:1042F00096028093BB0202C01092BB028091BC0266
:104300008230F1F5809137019091CA02890F809334
:104310001A0180911A01853020F080911A018B3F9B
:1043200018F085E080931A01809137012091C20234
:104330009091CA02820F890F8093B7028091210168
:104340002091B70290E0049730E0281739072CF04D
:104350008091210185508093B7028091B7028F3000
:1043600018F48FE08093B70280911A019091960221
:10437000890F80931A018091B7029091960208C02C
:104380008091370180931A01809137019091C20288
:10439000890F8093B70280918B0290918C0240919B
:1043A00031015091320120917F0230918002240F1F
:1043B000351F821B930B90932C0180932B018091CE
:1043C000030187BD8091C1022091030190E0049612
:1043D00030E0821793072CF0809103018550809381
:1043E000C102809103019091C102891B80938F02C9
:1043F0002091BF023091CF029091BC028091A10226
:1044000060E2269FA001112460E1369F90011124F3
:10441000242B282B34E0939FC0011124822B8093FE
:104420008E02E0918E028E2F90E0FC013197EA33EC
:10443000F105A0F4EE51FE4F0C94913C1092150141
:104440000DC080E209C082E007C080E105C081E2C2
:1044500003C082E101C081E08093150180911501C4
:10446000803109F4E3C058F48130C1F0823011F09A
:104470000C94B535109209011092080161C0803288
:1044800009F4C6C1813209F43DC2823111F00C94A5
:10449000B53510920901109208011AC11092090154
:1044A00010920801209108013091090180911801B2
:1044B00090E028173907C8F480911E0190911F01E0
:1044C0009C012F5F3F4F30931F0120931E01FC0181
:1044D000E75CFE4F108280910801909109010196DE
:1044E0009093090180930801DDCF10920901109289
:1044F000080143E0209108013091090180918B026D
:1045000090918C022817390710F00C94B5358091E2
:104510001E0190911F019C012F5F3F4F30931F019F
:1045200020931E01FC01E75CFE4F4083809108014F
:104530009091090101969093090180930801DACFC7
:1045400020910801309109018091180190E028170D
:104550003907C8F480911E0190911F019C012F5FC3
:104560003F4F30931F0120931E01FC01E75CFE4F7B
:1045700010828091080190910901019690930901A0
:1045800080930801DDCF109209011092080120915B
:104590000801309109018091310190913201281771
:1045A0003907C8F480911E0190911F019C012F5F73
:1045B0003F4F30931F0120931E01FC01E75CFE4F2B
:1045C0001082809108019091090101969093090150
:1045D00080930801DCCF109209011092080144E099
:1045E000209108013091090180917F029091800211
:1045F0002817390710F00C94B53580911E01909161
:104600001F019C012F5F3F4F30931F0120931E011C
:10461000FC01E75CFE4F4083809108019091090105
:1046200001969093090180930801DACF1092090155
:104630001092080120910801309109018091180120
:1046400090E028173907C8F480911E0190911F014E
:104650009C012F5F3F4F30931F0120931E01FC01EF
:10466000E75CFE4F1082809108019091090101964C
:104670009093090180930801DDCF109209011092F7
:10468000080145E0209108013091090180918B02D9
:1046900090918C022817390710F00C94B535809151
:1046A0001E0190911F019C012F5F3F4F30931F010E
:1046B00020931E01FC01E75CFE4F408380910801BE
:1046C0009091090101969093090180930801DACF36
:1046D00020910801309109018091180190E028177C
:1046E0003907C8F480911E0190911F019C012F5F32
:1046F0003F4F30931F0120931E01FC01E75CFE4FEA
:10470000108280910801909109010196909309010E
:1047100080930801DDCF109209011092080145E055
:10472000209108013091090180913101909132016D
:1047300028173907C8F480911E0190911F019C0130
:104740002F5F3F4F30931F0120931E01FC01E75C58
:10475000FE4F40838091080190910901019690934A
:10476000090180930801DCCF109209011092080121
:1047700046E0209108013091090180917F029091DB
:10478000800228173907C8F480911E0190911F01FB
:104790009C012F5F3F4F30931F0120931E01FC01AE
:1047A000E75CFE4F408380910801909109010196DA
:1047B0009093090180930801DCCF109209011092B7
:1047C000080145E0209108013091090180912B01F9
:1047D00090912C012817390710F00C94B535809171
:1047E0001E0190911F019C012F5F3F4F30931F01CD
:1047F00020931E01FC01E75CFE4F4083809108017D
:104800009091090101969093090180930801DACFF4
:1048100010920901109208012091080130910901BC
:104820008091180190E028173907C8F480911E0183
:1048300090911F019C012F5F3F4F30931F012093E8
:104840001E01FC01E75CFE4F1082809108019091EF
:10485000090101969093090180930801DDCF109220
:1048600009011092080120910801309109018091FD
:1048700031019091320128173907C8F480911E0147
:1048800090911F019C012F5F3F4F30931F01209398
:104890001E01FC01E75CFE4F10828091080190919F
:1048A000090101969093090180930801DCCF1092D1
:1048B00009011092080147E0209108013091090197
:1048C00080917F02909180022817390710F00C9494
:1048D000B53580911E0190911F019C012F5F3F4FC4
:1048E00030931F0120931E01FC01E75CFE4F4083C3
:1048F000809108019091090101969093090180939C
:104900000801DACF109209011092080120910801E4
:10491000309109018091180190E028173907C8F4F7
:1049200080911E0190911F019C012F5F3F4F30939A
:104930001F0120931E01FC01E75CFE4F1082809155
:104940000801909109010196909309018093080153
:10495000DDCF109209011092080143E02091080177
:104960003091090180913101909132012817390766
:10497000C8F480911E0190911F019C012F5F3F4F51
:1049800030931F0120931E01FC01E75CFE4F408322
:1049900080910801909109010196909309018093FB
:1049A0000801DCCF109209011092080148E0209123
:1049B00008013091090180917F02909180022817AF
:1049C0003907C8F480911E0190911F019C012F5F4F
:1049D0003F4F30931F0120931E01FC01E75CFE4F07
:1049E00040838091080190910901019690930901FB
:1049F00080930801DCCF109209011092080143E076
:104A0000209108013091090180912B0190912C0196
:104A10002817390710F00C94B53580911E0190913C
:104A20001F019C012F5F3F4F30931F0120931E01F8
:104A3000FC01E75CFE4F40838091080190910901E1
:104A400001969093090180930801DACF9091920228
:104A50008091000198130C94D332D5E0D0930001DB
:104A60001092920283B1847083B9811110C286B111
:104A7000817086B9882379F080917E028F5F809360
:104A80007E0280917E02843010F010927E028AE0D5
:104A900080930001FCC110927E02D093B602C1E067
:104AA000C0939D0286E0A82EA0921001C09335010C
:104AB000109230019CE3B92EB092270124E1F22E2E
:104AC000F092050188E790E09093A7028093A602F8
:104AD00082E380932001C09398023CE8C32ED12C3E
:104AE000D0928802C0928702C093C00210929302B3
:104AF0001092B2020EE110E01093A00200939F0208
:104B00008AE080932F0110931D0100931C01F09205
:104B1000970260919D0286E090E00E94A53C609122
:104B2000100188E090E00E94A53C609135018AE088
:104B300090E00E94A53C609130018CE090E00E94E2
:104B4000A53C609127018EE090E00E94A53C609119
:104B5000050180E190E00E94A53C6091A602709161
:104B6000A70282E190E00E94B73C6091200184E1BD
:104B700090E00E94A53C6091980286E190E00E943E
:104B8000A53C609187027091880288E190E00E94C4
:104B9000B73C6091C0028AE190E00E94A53C609120
:104BA00093028CE190E00E94A53C6091B2028EE1FC
:104BB00090E00E94A53C60919F027091A00280E26B
:104BC00090E00E94B73C60912F0182E290E00E9449
:104BD000A53C60911C0170911D0184E290E00E944F
:104BE000B73C6091970286E290E00E94A53CC0939A
:104BF000BE02A0929E02C093CF02D0939602B092C2
:104C0000C102F092180186E48093030144E6A42EC9
:104C1000B12CB0928C02A0928B02C0938D02D092E4
:104C2000D602C092D502C093BF021092CA0210925F
:104C3000AC028FE08093370154E1C52ED12CD09285
:104C40003201C09231018093C20288E290E09093D9
:104C5000800280937F026091BE020E94A53C609119
:104C60009E028AE290E00E94A53C6091CF028CE215
:104C700090E00E94A53C609196028EE290E00E9436
:104C8000A53C6091C10280E390E00E94A53C609148
:104C9000180182E390E00E94A53C6091030184E347
:104CA00090E00E94A53C60918B0270918C0286E39B
:104CB00090E00E94B73C60918D0288E390E00E94F2
:104CC000A53C6091D5027091D6028AE390E00E94E3
:104CD000B73C6091BF028CE390E00E94A53C6091DC
:104CE000CA028EE390E00E94A53C6091AC0280E491
:104CF00090E00E94A53C6091370182E490E00E9420
:104D0000A53C609131017091320184E490E00E94F1
:104D1000B73C6091C20286E490E00E94A53C60919D
:104D20007F027091800288E490E00E94B73C10926C
:104D30001B01D0937C0286E090E09093B1028093B7
:104D4000B002C093D4022AE530E0309312012093E0
:104D50001101109314010093130110939502009315
:104D60009402D092AE02C092AD02C0937A02D09368
:104D7000C4029093170180931601C093240186E921
:104D800090E09093260180932501B092C602A092F4
:104D9000C5021093860200938502D0922E01C09224
:104DA0002D0160911B018AE490E00E94A53C609176
:104DB0007C028CE490E00E94A53C6091B00270916E
:104DC000B1028EE490E00E94B73C6091D40280E58D
:104DD00090E00E94A53C609111017091120186E55E
:104DE00090E00E94B73C609113017091140188E536
:104DF00090E00E94B73C60919402709195028AE520
:104E000090E00E94B73C6091AD027091AE028CE5DB
:104E100090E00E94B73C60917A028EE590E00E949B
:104E2000A53C6091C40280E690E00E94A53C6091A0
:104E300016017091170182E690E00E94B73C6091E4
:104E4000240184E690E00E94A53C609125017091C8
:104E500026018AE690E00E94B73C6091C5027091FD
:104E6000C6028CE690E00E94B73C6091850270918A
:104E700086028EE690E00E94B73C60912D01709111
:104E80002E0180E790E00E94B73CF092000186B1CD
:104E9000817086B9811120C086B1827086B988235D
:104EA00061F08091B6028F5F8093B6028091B60266
:104EB000863078F01092B6020CC08091B602815014
:104EC0008093B6028091B602813F18F085E080930E
:104ED000B6028AE08093000186B1827086B98111A2
:104EE00004C08091C302806103C08091C3028F7EA1
:104EF0008093C30286B1847086B9811104C0809109
:104F0000C302886003C08091C302877F8093C3027D
:104F100086B1807186B9811104C08091C30284601A
:104F200003C08091C3028B7F8093C30286B18870D7
:104F300086B9811104C08091C302826003C0809150
:104F4000C3028D7F8093C30286B1807286B98111BE
:104F500004C08091C302816003C08091C3028E7F30
:104F60008093C3028091B602823009F4BFC238F444
:104F7000882379F0813009F4E8C00C94CD2F843077
:104F800009F4D5C408F4F8C3853009F48AC60C9432
:104F9000CD2FE091C3028E2F90E0FC013197EF31CD
:104FA000F10510F00C94CD2FE45EFD4F0C94913C74
:104FB00080917C02833030F48091B0029091B102F4
:104FC000449619C080917C02833031F48091B00204
:104FD0009091B1020A960FC080917C02843031F426
:104FE0008091B0029091B102029605C08091B0020A
:104FF0009091B10201969093B1028093B0022091FA
:10500000B0023091B1028091D2029091D302821706
:10501000930708F075C78091D2029091D3029093C4
:10502000B1028093B0026CC780917C028150809362
:105030007C0280917C02813F10F010927C0281E022
:10504000809338015DC780917C028F5F80937C02E2
:1050500080917C028A3018F089E080937C0281E0A4
:10506000809338014DC780917C02833030F4809169
:10507000B0029091B102449719C080917C028330B4
:1050800031F48091B0029091B1020A970FC08091E3
:105090007C02843031F48091B0029091B102029789
:1050A00005C08091B0029091B10201979093B10236
:1050B0008093B0028091B0029091B102893E9D4FE1
:1050C00008F41EC71092B1021092B00219C7909155
:1050D000D40281E089278093D40212C79091D40230
:1050E00081E089278093D4020BC79091D40281E09C
:1050F00089278093D40204C79091D40281E0892744
:105100008093D402FDC681E080933801F9C685E022
:1051100080937C0281E080933801F2C681E0809325
:10512000D402EEC681E08093D402EAC686E090E025
:105130009093B1028093B00285E080937C0281E07D
:105140008093D40280933801DBC6E091C3028E2F96
:1051500090E0FC013197EF31F10508F01EC7E55CE6
:10516000FD4F0C94913C8091110190911201019698
:105170009093120180931101C3C680911301909105
:1051800014010196909314018093130180911301EF
:10519000909114014091AD025091AE022091C50250
:1051A0003091C602840F951F2817390708F0A8C64A
:1051B00080911B018111A4C680911301909114016B
:1051C00001979093140180931301809113019091A2
:1051D000140120912D0130912E01820F931F909385
:1051E00014018093130181E080931B018091C5021B
:1051F0009091C6022091AD023091AE02821B930BBA
:105200009093C6028093C50210927A0279C680916B
:10521000130190911401019790931401809313014D
:105220008091130190911401893E9D4F20F01092BE
:105230001401109213018091C5029091C602409111
:105240002D0150912E012091130130911401840FF2
:10525000951F2817390708F053C620911B012130EC
:1052600009F04EC68091130190911401019690931C
:1052700014018093130180911301909114014091C6
:105280002D0150912E01841B950B90931401809356
:10529000130110921B018091C5029091C6024091AA
:1052A000AD025091AE02840F951F9093C602809379
:1052B000C50220937A0224C68091110190911201B7
:1052C00001979093120180931101809111019091A7
:1052D0001201089708F014C688E090E0909312013C
:1052E000809311010DC680911101909112010A96CF
:1052F000909312018093110103C680911301909144
:1053000014010A9690931401809313018091130164
:10531000909114014091AD025091AE022091C502CE
:105320003091C602840F951F2817390708F0E8C589
:1053300080911B018111E4C58091C5029091C60244
:105340002091AD023091AE02821B930B9093140119
:1053500080931301809113019091140120912D01EC
:1053600030912E01820F931F9093140180931301AB
:1053700081E080931B018091C5029091C60220912B
:10538000AD023091AE02821B930B9093C6028093C4
:10539000C50210927A02B4C5809113019091140154
:1053A0000A979093140180931301809113019091B7
:1053B0001401893E9D4F20F01092140110921301A8
:1053C0008091C5029091C60240912D0150912E010D
:1053D0002091130130911401840F951F281739076C
:1053E00008F08EC520911B01213009F089C58091FC
:1053F000C5029091C60240912D0150912E01840F5B
:10540000951F909314018093130180911301909143
:10541000140140912D0150912E01841B950B909306
:1054200014018093130110921B018091C502909189
:10543000C6024091AD025091AE02840F951F909329
:10544000C6028093C50220937A025AC58091110149
:10545000909112010A97909312018093110180910B
:10546000110190911201089740F0809111019091E3
:105470001201893E9D4F08F443C588E090E0909367
:105480001201809311013CC58AE590E090931201CE
:105490008093110135C58EE190E0909314018093C3
:1054A000130181E08093CD022BC58AE590E09093B3
:1054B00012018093110124C58EE190E090931401B4
:1054C0008093130181E08093CD021AC58AE590E0B4
:1054D00090931201809311018EE190E0909314015A
:1054E0008093130181E08093CD020AC5E091C3024D
:1054F0008E2F90E0FC013197EF31F10508F04DC59A
:10550000E65AFD4F0C94913C809194029091950243
:1055100001969093950280939402809194029091C9
:105520009502853F914008F4EBC4809194029091DC
:10553000950201979093950280939402E1C4809123
:10554000AD029091AE0201969093AE028093AD02AF
:105550008091AD029091AE028331914048F08091EC
:10556000AD029091AE0201979093AE028093AD028E
:1055700080911301909114014091AD025091AE02BF
:105580002091C5023091C602840F951F2817390754
:1055900008F0B6C480911B018111B2C48091AD02A4
:1055A0009091AE0201979093AE028093AD02A8C491
:1055B0008091AD029091AE0201979093AE028093DC
:1055C000AD028091AD029091AE020A9708F098C4A6
:1055D0008091AD029091AE0201969093AE028093BD
:1055E000AD028EC4809194029091950201979093A0
:1055F00095028093940280919402909195020F9766
:1056000008F07EC48FE090E090939502809394021E
:1056100077C480919402909195020A969093950296
:10562000809394028091940290919502853F9140DD
:1056300008F466C484EF91E09093950280939402FD
:105640005FC48091AD029091AE020A969093AE0233
:105650008093AD028091AD029091AE028331914072
:1056600030F082E191E09093AE028093AD028091A0
:105670001301909114014091AD025091AE0220911E
:10568000C5023091C602840F951F2817390708F00C
:1056900037C480911B01811133C48091C502909160
:1056A000C6022091130130911401821B930B909339
:1056B000AE028093AD0224C48091AD029091AE02FF
:1056C0000A979093AE028093AD028091AD029091C3
:1056D000AE020A9708F014C48AE090E09093AE02FC
:1056E0008093AD020DC480919402909195020A9727
:1056F00090939502809394028091940290919502E8
:105700000F9708F0FDC38FE090E09093950280938F
:105710009402F6C38EE190E09093950280939402F8
:10572000EFC384E190E09093AE028093AD0281E0FC
:105730008093CD02E5C38EE190E090939502809333
:105740009402DEC384E190E09093AE028093AD02B8
:1057500081E08093CD02D4C38EE190E090939502D6
:105760008093940284E190E09093AE028093AD0226
:1057700081E08093CD02C4C3E091C3028E2F90E0FC
:10578000FC013197EF31F10508F007C4E758FD4FF0
:105790000C94913C8091C402833030F480911601C6
:1057A00090911701449619C08091C402833031F45E
:1057B00080911601909117010A960FC08091C40242
:1057C000843031F48091160190911701029605C042
:1057D0008091160190911701019690931701809383
:1057E000160120911601309117018091AA02909123
:1057F000AB028217930708F083C38091AA029091AD
:10580000AB0290931701809316017AC38091C40272
:1058100081508093C4028091C402813F10F01092A5
:10582000C40281E08093C7026BC38091C4028F5F82
:105830008093C4028091C4028A3018F089E080937A
:10584000C40281E08093C7025BC38091C4028330AD
:1058500030F48091160190911701449719C08091FE
:10586000C402833031F480911601909117010A9798
:105870000FC08091C402843031F480911601909160
:105880001701029705C080911601909117010197A9
:105890009093170180931601809116019091170142
:1058A000893E9D4F08F42CC31092170110921601E7
:1058B00027C39091240181E089278093240120C38C
:1058C0009091240181E089278093240119C390914C
:1058D000240181E089278093240112C3909124013F
:1058E00081E08927809324010BC381E08093C70264
:1058F00007C385E08093C40281E08093C70200C3A0
:1059000081E080932401FCC281E080932401F8C2ED
:1059100086E090E0909317018093160185E08093D4
:10592000C40281E0809324018093C702E9C2E09120
:10593000C3028E2F90E0FC013197EF31F10508F0A2
:105940002CC3E856FD4F0C94913C80912501909119
:10595000260101969093260180932501D1C2809162
:10596000C5029091C60201969093C6028093C5022B
:105970008091C5029091C60240912D0150912E0157
:105980002091130130911401840F951F28173907B6
:1059900008F0B6C280917A028111B2C28091C5022C
:1059A0009091C60201979093C6028093C5028091A0
:1059B000C5029091C6022091AD023091AE02820FD5
:1059C000931F9093C6028093C50281E080937A0270
:1059D000809113019091140120912D0130912E019D
:1059E000821B930B909314018093130110921B015F
:1059F00087C28091C5029091C60201979093C6021A
:105A00008093C5028091C5029091C602893E9D4F48
:105A100020F01092C6021092C5028091130190915D
:105A200014014091AD025091AE022091C502309117
:105A3000C602840F951F2817390708F061C220910C
:105A40007A02213009F05CC28091C5029091C602B1
:105A500001969093C6028093C5028091C5029091F1
:105A6000C6024091AD025091AE02841B950B9093FB
:105A7000C6028093C50210927A0280911301909120
:105A8000140140912D0150912E01840F951F909388
:105A900014018093130120931B0132C280912501D0
:105AA0009091260101979093260180932501809182
:105AB000250190912601089708F022C288E090E025
:105AC00090932601809325011BC28091250190911E
:105AD00026010A96909326018093250111C2809198
:105AE000C5029091C6020A969093C6028093C502A1
:105AF0008091C5029091C60240912D0150912E01D6
:105B00002091130130911401840F951F2817390734
:105B100008F0F6C180917A028111F2C180911301DF
:105B20009091140120912D0130912E01821B930B35
:105B30009093C6028093C5028091C5029091C602DF
:105B40002091AD023091AE02820F931F9093C60256
:105B50008093C50281E080937A0280911301909135
:105B6000140120912D0130912E01821B930B9093F3
:105B700014018093130110921B01C2C18091C502D0
:105B80009091C6020A979093C6028093C5028091B5
:105B9000C5029091C602893E9D4F20F01092C60228
:105BA0001092C50280911301909114014091AD02B1
:105BB0005091AE022091C5023091C602840F951F0C
:105BC0002817390708F09CC120917A02213009F08A
:105BD00097C180911301909114014091AD025091B1
:105BE000AE02840F951F9093C6028093C5028091E8
:105BF000C5029091C6024091AD025091AE02841B45
:105C0000950B9093C6028093C50210927A02809100
:105C100013019091140140912D0150912E01840F98
:105C2000951F909314018093130120931B0168C169
:105C300080912501909126010A97909326018093E7
:105C400025018091250190912601089740F08091CF
:105C5000250190912601893E9D4F08F451C188E0AD
:105C600090E090932601809325014AC186E990E057
:105C7000909326018093250143C186E990E090939B
:105C80002601809325013CC186E990E0909326018E
:105C90008093250184E690E09093C6028093C5022C
:105CA0002CC1E091C3028E2F90E0FC013197EF31BF
:105CB000F10508F072C1E954FD4F0C94913C8091BC
:105CC00085029091860201969093860280938502C8
:105CD0008091850290918602853F914008F410C121
:105CE000809185029091860201979093860280931D
:105CF000850206C180912D0190912E01019690930D
:105D00002E0180932D0180912D0190912E018331E0
:105D1000914048F080912D0190912E010197909330
:105D20002E0180932D018091C5029091C602409171
:105D30002D0150912E012091130130911401840FF7
:105D4000951F2817390708F0DBC080917A0281116E
:105D5000D7C080912D0190912E01019790932E0133
:105D600080932D01CDC080912D0190912E0101973E
:105D700090932E0180932D0180912D0190912E0101
:105D80000A9708F0BDC080912D0190912E010196D7
:105D900090932E0180932D01B3C080918502909144
:105DA00086020197909386028093850280918502F6
:105DB000909186020F9708F0A3C08FE090E0909337
:105DC0008602809385029CC0809185029091860214
:105DD0000A96909386028093850280918502909125
:105DE0008602853F914008F48BC084EF91E0909348
:105DF00086028093850284C080912D0190912E01AE
:105E00000A9690932E0180932D0180912D019091FF
:105E10002E018331914030F082E191E090932E0188
:105E200080932D018091C5029091C60240912D0171
:105E300050912E012091130130911401840F951F70
:105E40002817390708F05CC080917A02811158C088
:105E500080911301909114012091C5023091C602E6
:105E6000821B930B90932E0180932D0149C080914A
:105E70002D0190912E010A9790932E0180932D0170
:105E800080912D0190912E010A97D0F58AE090E043
:105E900090932E0180932D0133C0809185029091C3
:105EA00086020A97909386028093850280918502EC
:105EB000909186020F9720F58FE090E090938602F4
:105EC000809385021DC08EE190E0909386028093BE
:105ED000850216C08EE190E0909386028093850241
:105EE0000FC08EE190E0909386028093850284E15A
:105EF00090E090932E0180932D0181E08093BD026C
:105F00008AE049C010921B0166E070E07093B10214
:105F10006093B00295E090937C0281E08093D4027C
:105F2000809338012AE530E030931201209311016B
:105F30002EE130E030931401209313013093950249
:105F40002093940244E150E05093AE024093AD029E
:105F500080937A0270931701609316019093C402A4
:105F6000809324018093C70286E990E090932601F4
:105F70008093250184E690E09093C6028093C50249
:105F8000309386022093850250932E0140932D0179
:105F90001092B60284E1809300018091CD028823A3
:105FA00009F491C08091C5029091C60240912D01E3
:105FB00050912E012091130130911401840F951FEF
:105FC0008217930730F481E080931B0110927A02CC
:105FD00078C02091C5023091C60280911301909142
:105FE00014012817390768F52091C5023091C602BF
:105FF00060912D0170912E018091130190911401F7
:106000004091AD025091AE02260F371F840F951FAD
:1060100028173907B8F581E080931B0110927A02A6
:106020008AE090E090932E0180932D0180911301DE
:106030009091140120912D0130912E01821B930B20
:1060400036C02091C5023091C60280911301909113
:1060500014014091AD025091AE02840F951F281794
:10606000390750F52091C5023091C60260912D018B
:1060700070912E0180911301909114014091AD0215
:106080005091AE0210921B0181E080937A028AE067
:1060900090E090932E0180932D01809113019091B7
:1060A00014012091AD023091AE02820F931F9093A4
:1060B000C6028093C50205C010921B0181E0809347
:1060C0007A021092CD028091BD02882309F493C018
:1060D00080911301909114014091AD025091AE0254
:1060E0002091C5023091C602840F951F8217930735
:1060F00030F410921B0181E080937A027AC02091E3
:106100001301309114018091C5029091C6022817A5
:10611000390788F420911301309114016091AD0288
:106120007091AE028091C5029091C60240912D01FE
:1061300050912E0129C02091C5023091C602809154
:106140001301909114014091AD025091AE02840F61
:10615000951F2817390708F047C02091C5023091D4
:10616000C60260912D0170912E01809113019091D2
:1061700014014091AD025091AE02260F371F840FDB
:10618000951F28173907D0F410921B0181E08093E6
:106190007A028AE090E09093AE028093AD02809103
:1061A000C5029091C6022091AD023091AE02821BD1
:1061B000930B90931401809313011BC081E0809393
:1061C0001B0110927A028AE090E09093AE028093D5
:1061D000AD028091C5029091C60220912D013091AF
:1061E0002E01820F931FE5CF81E080931B01109257
:1061F0007A021092BD0280917A02882309F475C058
:106200008091C5029091C60220912D0130912E01FE
:10621000820F931F8331914008F4D9C02091C502A9
:106220003091C60282E191E0821B930B90932E0184
:1062300080932D0180912D0190912E01893E9D4FDB
:1062400030F480912D0190912E010A97C8F48AE0D4
:1062500090E090932E0180932D018091C502909142
:10626000C60220912D0130912E01820F931F8331A0
:10627000914030F088E091E09093C6028093C5028F
:1062800080911301909114014091AD025091AE02A2
:106290002091C5023091C602840F951F2817390737
:1062A00008F095C08091C5029091C6022091AD0280
:1062B0003091AE02821B930B9093140180931301D3
:1062C0008091130190911401893E9D4F08F47FC085
:1062D00010921401109213018091C5029091C60290
:1062E0009093AE028093AD0272C0809113019091A1
:1062F00014012091AD023091AE02820F931F8331C1
:10630000914008F464C0209113013091140182E19E
:1063100091E0821B930B9093AE028093AD0280912B
:10632000AD029091AE02893E9D4F30F48091AD0256
:106330009091AE020A97C8F48AE090E09093AE0282
:106340008093AD0280911301909114012091AD02D0
:106350003091AE02820F931F8331914030F088E07C
:1063600091E090931401809313018091C502909164
:10637000C60240912D0150912E01209113013091C0
:106380001401840F951F2817390708F58091130110
:106390009091140120912D0130912E01821B930BBD
:1063A0009093C6028093C5028091C5029091C60267
:1063B000893E9D4F60F01092C6021092C5028091F6
:1063C00013019091140190932E0180932D018091DF
:1063D0001101909112012091940230919502820F47
:1063E000931F853E924060F0209194023091950277
:1063F00084EE92E0821B930B909312018093110123
:10640000809125019091260120918502309186028C
:10641000820F931F853E924060F02091850230915B
:10642000860284EE92E0821B930B90932601809368
:106430002501E0917C028E2F90E08A30910530F5A5
:10644000FC01EA52FD4F0C94913C88E191E01AC0A6
:1064500088E790E017C080E590E014C088E290E003
:1064600011C088E190E00EC08CE090E00BC088E0A5
:1064700090E008C086E090E005C085E090E002C0B2
:1064800084E090E09093D3028093D202809138010F
:10649000813061F5E0917C028E2F90E08A30910589
:1064A00018F5FC01E052FD4F0C94913C8CE890E013
:1064B00017C08CE390E014C088E290E011C084E142
:1064C00090E00EC08CE090E00BC086E090E008C049
:1064D00084E090E005C083E090E002C082E090E0BC
:1064E0009093B1028093B00210923801E091C402FF
:1064F0008E2F90E08A30910530F5FC01E651FD4F7A
:106500000C94913C88E191E01AC088E790E017C0B4
:1065100080E590E014C088E290E011C088E190E04E
:106520000EC08CE090E00BC088E090E008C086E0F0
:1065300090E005C085E090E002C084E090E0909398
:10654000AB028093AA028091C702813061F5E0918D
:10655000C4028E2F90E08A30910518F5FC01EC50B2
:10656000FD4F0C94913C8CE890E017C08CE390E0D8
:1065700014C088E290E011C084E190E00EC08CE08D
:1065800090E00BC086E090E008C084E090E005C099
:1065900083E090E002C082E090E090931701809346
:1065A00016011092C702809192028F5F809392022F
:1065B000809182029091830201969093830280934E
:1065C000820220918202309183028091D2029091C6
:1065D000D3022817390720F010928302109282020A
:1065E00020918202309183028091B0029091B10299
:1065F0002817390720F481E08093060102C0109229
:10660000060180910D0190910E01019690930E016B
:1066100080930D0120910D0130910E018091AA020D
:106620009091AB022817390720F010920E011092BA
:106630000D0120910D0130910E0180911601909174
:1066400017012817390720F481E08093790202C0EE
:106650001092790280911101909112019093290179
:106660008093280180911101909112012091940250
:1066700030919502820F931F90938A028093890232
:10668000809125019091260190932301809322010E
:1066900080912501909126012091850230918602FA
:1066A000820F931F9093DA028093D90280911B018D
:1066B000882369F080911301909114014091C502E3
:1066C0005091C60220912D0130912E010CC0809175
:1066D000C5029091C602409113015091140120917E
:1066E000AD023091AE02240F351F821B930B9093A5
:1066F000CC028093CB028091D40290910601892331
:1067000080930601809124019091790289238093DE
:106710007902809179029091060120911B0130E26B
:10672000839FA001112460E1969FC0011124842B56
:10673000822B80930201809102018131D1F038F4E3
:10674000813089F080F08031B1F481E112C0813272
:1067500069F018F4803251F00EC0803349F0813373
:1067600051F481E206C01092A20205C082E201C08B
:1067700082E18093A2028091A202823109F4B0C02A
:1067800040F4813109F0F1C1109209011092080121
:106790000BC0813209F447C1823209F0E6C1109280
:1067A0000901109208014EC02091080130910901A1
:1067B000809113019091140128173907C8F4809132
:1067C0001E0190911F019C012F5F3F4F30931F01CD
:1067D00020931E01FC01E75CFE4F108280910801AE
:1067E0009091090101969093090180930801DCCFF3
:1067F000109209011092080141E0209108013091A6
:1068000009018091AD029091AE022817390708F076
:10681000ACC180911E0190911F019C012F5F3F4FE1
:1068200030931F0120931E01FC01E75CFE4F408363
:10683000809108019091090101969093090180933C
:106840000801DBCF20910801309109018091C50238
:106850009091C60228173907C8F480911E019091C3
:106860001F019C012F5F3F4F30931F0120931E019A
:10687000FC01E75CFE4F10828091080190910901B4
:1068800001969093090180930801DCCF10920901D1
:106890001092080142E02091080130910901809195
:1068A0002D0190912E012817390708F05EC18091C3
:1068B0001E0190911F019C012F5F3F4F30931F01DC
:1068C00020931E01FC01E75CFE4F4083809108018C
:1068D0009091090101969093090180930801DBCF03
:1068E00010920901109208012091080130910901CC
:1068F000809113019091140128173907C8F48091F1
:106900001E0190911F019C012F5F3F4F30931F018B
:1069100020931E01FC01E75CFE4F1082809108016C
:106920009091090101969093090180930801DCCFB1
:10693000109209011092080141E020910801309164
:1069400009018091AD029091AE0228173907C8F471
:1069500080911E0190911F019C012F5F3F4F30934A
:106960001F0120931E01FC01E75CFE4F40838091D4
:106970000801909109010196909309018093080103
:10698000DCCF10920901109208012091080130918A
:1069900009018091CB029091CC0228173907C8F4E5
:1069A00080911E0190911F019C012F5F3F4F3093FA
:1069B0001F0120931E01FC01E75CFE4F10828091B5
:1069C00008019091090101969093090180930801B3
:1069D000DCCF109209011092080142E020910801D9
:1069E0003091090180912D0190912E0128173907CE
:1069F00008F0BBC080911E0190911F019C012F5F88
:106A00003F4F30931F0120931E01FC01E75CFE4FB6
:106A100040838091080190910901019690930901AA
:106A200080930801DBCF1092090110920801209198
:106A30000801309109018091C5029091C602281782
:106A40003907C8F480911E0190911F019C012F5FAE
:106A50003F4F30931F0120931E01FC01E75CFE4F66
:106A6000108280910801909109010196909309018B
:106A700080930801DCCF109209011092080142E0D6
:106A8000209108013091090180912D0190912E01F2
:106A900028173907C8F480911E0190911F019C01AD
:106AA0002F5F3F4F30931F0120931E01FC01E75CD5
:106AB000FE4F4083809108019091090101969093C7
:106AC000090180930801DCCF10920901109208019E
:106AD00020910801309109018091CB029091CC0264
:106AE00028173907C8F480911E0190911F019C015D
:106AF0002F5F3F4F30931F0120931E01FC01E75C85
:106B0000FE4F1082809108019091090101969093A7
:106B1000090180930801DCCF10920901109208014D
:106B200041E020910801309109018091AD029091DE
:106B3000AE0228173907C8F480911E0190911F01F9
:106B40009C012F5F3F4F30931F0120931E01FC01DA
:106B5000E75CFE4F40838091080190910901019606
:106B60009093090180930801DCCF80911E019091E0
:106B70001F018331914080F480911E0190911F018B
:106B80009C012F5F3F4F30931F0120931E01FC019A
:106B9000E75CFE4F1082E9CF10921F0110921E0198
:106BA0001092A802809100018A3028F010920C0106
:106BB00010920B0109C080910B0190910C0101967C
:106BC00090930C0180930B0180910B0190910C012B
:106BD0008835924008F454C160919D0286E090E0AF
:106BE0000E94A53C6091100188E090E00E94A53CC5
:106BF000609135018AE090E00E94A53C60913001EF
:106C00008CE090E00E94A53C609127018EE090E02E
:106C10000E94A53C6091050180E190E00E94A53CA6
:106C20006091A6027091A70282E190E00E94B73CB9
:106C30006091200184E190E00E94A53C609198025F
:106C400086E190E00E94A53C6091870270918802E5
:106C500088E190E00E94B73C6091C0028AE190E038
:106C60000E94A53C609193028CE190E00E94A53CBB
:106C70006091B2028EE190E00E94A53C60919F027B
:106C80007091A00280E290E00E94B73C60912F01D9
:106C900082E290E00E94A53C60911C0170911D0170
:106CA00084E290E00E94B73C6091970286E290E017
:106CB0000E94A53C6091BE0288E290E00E94A53C43
:106CC00060919E028AE290E00E94A53C6091CF0212
:106CD0008CE290E00E94A53C609196028EE290E0EA
:106CE0000E94A53C6091C10280E390E00E94A53C17
:106CF0006091180182E390E00E94A53C609103013D
:106D000084E390E00E94A53C60918B0270918C021C
:106D100086E390E00E94B73C60918D0288E390E0AA
:106D20000E94A53C6091D5027091D6028AE390E062
:106D30000E94B73C6091BF028CE390E00E94A53CAA
:106D40006091CA028EE390E00E94A53C6091AC0283
:106D500080E490E00E94A53C6091370182E490E0DD
:106D60000E94A53C609131017091320184E490E071
:106D70000E94B73C6091C20286E490E00E94A53C6C
:106D800060917F027091800288E490E00E94B73C9D
:106D900060911B018AE490E00E94A53C60917C0216
:106DA0008CE490E00E94A53C6091B0027091B10229
:106DB0008EE490E00E94B73C6091D40280E590E0C0
:106DC0000E94A53C609111017091120186E590E04E
:106DD0000E94B73C609113017091140188E590E026
:106DE0000E94B73C60919402709195028AE590E010
:106DF0000E94B73C6091AD027091AE028CE590E0CC
:106E00000E94B73C60917A028EE590E00E94A53C1A
:106E10006091C40280E690E00E94A53C609116015A
:106E20007091170182E690E00E94B73C60912401C6
:106E300084E690E00E94A53C6091250170912601B6
:106E40008AE690E00E94B73C6091C5027091C6024C
:106E50008CE690E00E94B73C6091850270918602BA
:106E60008EE690E00E94B73C60912D0170912E015A
:106E700080E790E00E94B73C10920C0110920B0149
:106E80008091B602823089F038F4882359F081303D
:106E9000E1F55998589A39C0843071F048F085303E
:106EA000F9F033C08BB18C7F05C0599A58982DC02A
:106EB0008BB183608BB929C080910701863018F4AB
:106EC0008BB1836002C08BB18C7F8BB9809107013D
:106ED0008F5F80930701809107018C30B0F013C061
:106EE00080910701833018F48BB1836002C08BB1AD
:106EF0008C7F8BB9809107018F5F80930701809110
:106F00000701863010F01092070180917E028130D7
:106F100059F038F0823059F0833069F485B18360DC
:106F200009C085B18C7F06C0299A289804C0299889
:106F3000289A01C085B980E094E090938500809301
:106F4000840080916F00866080936F00FF91EF91C5
:106F5000DF91CF91BF91AF919F918F917F916F9171
:106F60005F914F913F912F911F910F91FF90DF9073
:106F7000CF90BF90AF900F900FBE0F901F901895BD
:106F80005C9A18955C98189578941F920F920FB69A
:106F90000F9211248F939F93AF93BF93EF93FF931F
:106FA000109285001092840080918F0286BDE0913E
:106FB0001E01F0911F01E75CFE4FE0818E2F90E0F3
:106FC0008930910508F0D0C0FC01E250FD4F0C94CF
:106FD000913C8091280190912901909389008093A0
:106FE00088008091890290918A020CC080912201D0
:106FF0009091230190938900809388008091D90219
:107000009091DA0290938B0080938A00ADC080E06B
:1070100094E09093850080938400A6C080E094E083
:10702000909385008093840096B580918F02891794
:10703000D8F386B58A30E8F386B58B30E8F796B595
:107040008091BB029817D8F35C9A86B58B30E8F72D
:107050008AC080E094E0909385008093840096B588
:1070600080918F028917D8F386B58A30E8F386B508
:107070008B30E8F796B580911A019817D8F35C9A8F
:1070800096B58091B7029817D8F36DC080E094E070
:10709000909385008093840096B580918F02891724
:1070A000D8F35C9A96B5809121019817D8F35BC00C
:1070B00080E094E0909385008093840096B5809161
:1070C0008F028917D8F35C9A96B5809121019817A1
:1070D000D8F35C9886B58B30E8F796B580911A01A5
:1070E0009817D8F35C9A96B58091B7029817D8F3A1
:1070F0003AC080E094E0909385008093840096B538
:1071000080918F028917D8F396B580911A0198174C
:10711000D8F35C9A96B58091B7029817D8F323C03C
:1071200080E094E0909385008093840096B58091F0
:107130008F028917D8F396B580911A019817D8F362
:107140005C9A96B58091B7029817D8F35C9886B58B
:107150008B30E8F796B58091BB029817D8F35C9A0C
:1071600086B58B30E8F75C988091A80291E0980F83
:107170009093A802833059F41092A80280911E01C6
:1071800090911F01019690931F0180931E01FF9122
:10719000EF91BF91AF919F918F910F900FBE0F9084
:1071A0001F901895549A579A84B1836084B98AB114
:1071B00083608AB988B18F6388B92A9A80918100E7
:1071C0008560809381005F9A0E942F038823E1F3FA
:1071D0005F988091A502882321F0809169008360E7
:1071E00008C0809169008260809369008091690085
:1071F0008E7F8093690080919C02882321F080918A
:1072000069008C6008C08091690088608093690083
:10721000809169008B7F80936900809181008B7FD2
:107220008093810084B5826084BD85B5816085BD11
:1072300086E090E00E94973C80939D0280919D02A1
:10724000863018F081E080939D0288E090E00E94F3
:10725000973C8093100180911001893118F086E0ED
:10726000809310018AE090E00E94973C8093350162
:1072700080913501823018F081E0809335018CE0F7
:1072800090E00E94973C80933001809130018531DD
:1072900010F0109230018EE090E00E94973C8093B5
:1072A000270180912701883020F080912701813FBC
:1072B00018F08CE38093270180E190E00E94973CD6
:1072C0008093050180910501813F18F084E180934E
:1072D000050182E190E00E949F3C9093A702809379
:1072E000A6028091A6029091A7024E9738F0809155
:1072F000A6029091A702853F914030F088E790E088
:107300009093A7028093A60284E190E00E94973CAC
:107310008093200180912001893120F0809120010B
:107320008A3818F082E38093200186E190E00E9481
:10733000973C8093980280919802863018F081E003
:107340008093980288E190E00E949F3C909388028D
:10735000809387028091870290918802813E9140BC
:1073600030F08CE890E090938802809387028AE165
:1073700090E00E94973C8093C0028091C0028230CE
:1073800018F081E08093C0028CE190E00E94973C6D
:107390008093930280919302873F24F0809193021F
:1073A0008A3014F0109293028EE190E00E94973C94
:1073B0008093B2028091B202813A10F01092B20230
:1073C00080E290E00E949F3C9093A00280939F02F5
:1073D00080919F029091A002853F914030F08EE114
:1073E00090E09093A00280939F0282E290E00E943E
:1073F000973C80932F0180912F018A3818F08AE002
:1074000080932F0184E290E00E949F3C90931D01A5
:1074100080931C0180911C0190911D010F9738F001
:1074200080911C0190911D01853F914030F08EE1CB
:1074300090E090931D0180931C0186E290E00E94F1
:10744000973C80939702809197028A3020F0809138
:1074500097028A3818F084E18093970288E290E0DE
:107460000E94973C8093BE028091BE02863018F045
:1074700081E08093BE028AE290E00E94973C809374
:107480009E0280919E02893118F086E080939E02D0
:107490008CE290E00E94973C8093CF028091CF02D3
:1074A000823018F081E08093CF028EE290E00E945B
:1074B000973C8093960280919602893218F085E07D
:1074C0008093960280E390E00E94973C8093C102F3
:1074D0008091C102883020F08091C102813F18F074
:1074E0008CE38093C10282E390E00E94973C8093FA
:1074F000180180911801813F18F084E180931801F0
:1075000084E390E00E94973C809303018091030103
:107510008C3320F0809103018B3F18F086E4809338
:10752000030186E390E00E949F3C90938C0280933D
:107530008B0280918B0290918C02C29738F08091DF
:107540008B0290918C028331914030F084E690E080
:1075500090938C0280938B0288E390E00E94973C8A
:1075600080938D0280918D02863018F081E08093A7
:107570008D028AE390E00E949F3C9093D602809314
:10758000D5028091D5029091D602813E914030F093
:107590008CE890E09093D6028093D5028CE390E043
:1075A0000E94973C8093BF028091BF02823018F006
:1075B00081E08093BF028EE390E00E94973C80932D
:1075C000CA028091CA02873F24F08091CA028A30A1
:1075D00014F01092CA0280E490E00E94973C8093DD
:1075E000AC028091AC02813A10F01092AC0282E4BD
:1075F00090E00E94973C809337018091370185305D
:1076000020F080913701813F18F08FE0809337019F
:1076100084E490E00E949F3C90933201809331017A
:1076200080913101909132018B3E910530F084E1DF
:1076300090E0909332018093310186E490E00E94C3
:10764000973C8093C2028091C2028A3020F08091E0
:10765000C202813F18F08FE08093C20288E490E07C
:107660000E949F3C9093800280937F0280917F02D2
:1076700090918002449738F080917F02909180022F
:107680008331914030F088E290E0909380028093C3
:107690007F028AE490E00E94973C80931B018091D6
:1076A0001B01823010F010921B018CE490E00E94CC
:1076B000973C80937C0280917C028A3018F085E0B0
:1076C00080937C028EE490E00E949F3C9093B102F4
:1076D0008093B0028091B0029091B10289319140C3
:1076E00030F086E090E09093B1028093B00280E5A4
:1076F00090E00E94973C8093D4028091D402823023
:1077000018F081E08093D40286E590E00E949F3CCF
:1077100090931201809311018091110190911201B7
:10772000089738F08091110190911201853E9240A6
:1077300030F08AE590E0909312018093110188E582
:1077400090E00E949F3C90931401809313018091DC
:107750001301909114018331914030F08EE190E05B
:1077600090931401809313018AE590E00E949F3C5E
:107770009093950280939402809194029091950247
:107780000F9738F08091940290919502853F914037
:1077900030F08EE190E090939502809394028CE516
:1077A00090E00E949F3C9093AE028093AD02809146
:1077B000AD029091AE020A9738F08091AD0290919F
:1077C000AE028331914030F084E190E09093AE02BC
:1077D0008093AD028EE590E00E94973C80937A0200
:1077E00080917A02823018F081E080937A0280E6FC
:1077F00090E00E94973C8093C4028091C4028A303A
:1078000018F085E08093C40282E690E00E949F3CDD
:1078100090931701809316018091160190911701A2
:107820008931914030F086E090E090931701809389
:10783000160184E690E00E94973C80932401809199
:107840002401823018F081E0809324018AE690E0E0
:107850000E949F3C909326018093250180912501F1
:1078600090912601089738F080912501909126018A
:10787000853E924030F086E990E090932601809317
:1078800025018CE690E00E949F3C9093C602809375
:10789000C5028091C5029091C6028331914030F0BB
:1078A00084E690E09093C6028093C5028EE690E055
:1078B0000E949F3C9093860280938502809185026E
:1078C000909186020F9738F0809185029091860200
:1078D000853F914030F08EE190E090938602809356
:1078E000850280E790E00E949F3C90932E01809358
:1078F0002D0180912D0190912E010A9738F08091F1
:107900002D0190912E018331914030F084E190E07F
:1079100090932E0180932D018DB383608DBB78945D
:10792000FFCFEE0FFF1F0590F491E02D0994F99918
:10793000FECF92BD81BDF89A992780B50895A8E140
:10794000B0E042E050E00C94BF3C262FF999FECF06
:1079500092BD81BDF89A019700B4021639F01FBAA2
:1079600020BD0FB6F894FA9AF99A0FBE08950196C1
:10797000272F0E94A63C0C94A53CDC01CB01FC0106
:10798000F999FECF06C0F2BDE1BDF89A319600B478
:0E7990000D9241505040B8F70895F894FFCF83
:02799E000500E2
:00000001FF
